:100000000C94512C0C94022D0C94022D0C94022D66
:100010000C94022D0C94022D0C94022D0C94022DA4
:100020000C94022D0C94022D0C94022D0C94022D94
:100030000C94022D0C94ED430C94022D0C94022D83
:100040000C94022D0C94022D0C94022D0C94022D74
:100050000C94022D0C94022D0C94022D0C94022D64
:100060000C94022D0C94022D0C94022D0C94022D54
:100070000000000000000000000000000000000080
:100080000000000000000000000000000000000070
:100090000000000000000000000000000000000060
:1000A0000000000000000000000000000000000050
:1000B0000000000000000000000000000000000040
:1000C00000000049000000495252000052525C2DCD
:1000D0000000000000000000000000000000000020
:1000E0000040000000494A52004952525B1C5253E2
:1000F0001C25241B2425251B0A0A2D1C12120A0A62
:100100000000000000000000404949494949525B95
:100110005B5B525B1C1C1312241C12090909120997
:100120000909090A0A0A0A0A0A13120A0A12130A10
:100130000000000000009252525252521312130952
:10014000001C0A1212401B65090A0009241B120038
:1001500000251C1C010025241C1C0024252424240B
:100160000000000000005249494000001B135249A2
:100170004900641C1C5B4A481C651C2552491C1C18
:10018000652464491C1C652564491C1C6D2E5C4952
:100190000000000000000000000000490000000016
:1001A000535200000053522500004A5225250000FA
:1001B0005B251300005B53000A1C095B1C657F373D
:1001C0004052522E2E1C525C2E251B1324251C1C23
:1001D00012002525120000121B0000132E37001BF1
:1001E00037372E2E37372E2E2E2E2E2E6E6E6E1C5D
:1001F0001313120009131200001213130012251C0E
:1002000013132E371C131313361C131B1B1B251320
:100210001C1C1B1B1B1C1C1C1C1C1C1C1C1C1C132A
:100220001312121313001313131C000913131C01D0
:100230000037131C13002E2E1C1C001C772E2500CB
:10024000137F251C010A37241C1C0A2E25250900B2
:10025000132E242525252E252525252525252D2E3E
:10026000251B2E2E251C1325251C1C1C1C011C1CAB
:100270001300011C0A000165775C016E7F6E521B42
:1002800025256D1C524925251C1353001C1C1C528E
:100290004A001B135B5B000009525C0000005B5CC2
:1002A000000000001B000000000000000000000033
:1002B000135B7F776E6E136577766E6E1B65777650
:1002C00076761B5BBF76B67609136DBFB7B6001B9B
:1002D000125C76BF0000121B125B00000000090ACE
:1002E0006E6E6E77241C6E6E77251C1C6E776E1CEE
:1002F0001C1C76761C1C2425B765646D6D1B766D01
:100300006D5B09125B5C5B125B641213131B1212B0
:100310001C1C1C1C1C241C1C242525242425251BDA
:1003200000002513000064BF00096EBFBF6D6EBFE3
:100330006D5B12135B12131209000901000000002B
:100340002E1C0900096E010009767F7F12777F7FDE
:100350006412BF775B121B095B121B0900001B09AB
:10036000000000000000000000000000000000008D
:100370007F7F5313130064121B0100001B12000047
:10038000000000000000000000000000000000006D
:10039000000000000000000000000000000000005D
:1003A0000000000000002600000026002F000000D2
:1003B0002F00370000003700FF000000FF00BF00E3
:1003C0000000BF00370000370000002626000000B4
:1003D000000000000000262626262600000000005F
:1003E0002F000000003700000000FF00000000BFE9
:1003F0000000000037000000000026262626260008
:100400000000000000002626262626002F000000FF
:100410000000370000000000FFFFFFFF0000BF00EA
:1004200000000000370000000000262626262600D7
:100430000000000000002626262600002F000000F5
:100440002F00370000003700FFFFFFFF0000BF0054
:100450000000BF00370000003700262626260000D7
:10046000000000000000000026262600002F0000EB
:100470002F00370000003700FF000000FF00BF0022
:100480000000BF00370000370000262626000000CD
:100490000000000000002600000026002F000000E1
:1004A0002F000037003700000000FF00000000BFF1
:1004B00000BF0000370000003700260000002600C3
:1004C000000000000000000000000000000000002C
:1004D000000000000000000000000000000000001C
:1004E0000000009B000000529BA400005B9B6D7706
:1004F00000000000000000000000000000000000FC
:10050000005B000000E4F6FF099BEDF6FFBFA4AD21
:10051000BFBFBFBF767F7FB7B7BF7F766EB7B7BFAE
:1005200000000000000000005BB6F6F6F6FFFFFFDB
:10053000FFBFFFFFFFBFBFAEFFFFFFB7AD65FFFF10
:10054000B7B6AD65FFFFBFB7AE6EFFFFBFB7B7650C
:10055000000000000000F6F6EDEDADA4B66D6D5C98
:10056000526E6565655265765C5C52536E246552C9
:10057000526E25255B52772D2525526E6E2D252531
:10058000000000000000A49B9B4900006564A49B40
:1005900092006D2525649349656E652E9B52242536
:1005A0006D25655225246D2D655225256E2E6452CC
:1005B00000000000000000000000004A00000000F1
:1005C0005B9B0000005B5B2D0000525B2E2E000148
:1005D0005B2D1C01005C5B014A654A5B1C6E7F77EA
:1005E000495B9B77776D5B65776E65656D2D25251E
:1005F0005C522E25130949641C09095C7F7F091C84
:100600007F7F777F777F77777F7F7776777F7F6E44
:10061000656E6EA4B6FF655BA4B7BFFF526DBFBF2A
:10062000BFFF7FBFBFBFBFFFBFBFB7BFFFFF7FB76A
:10063000BFBFFFFF6EB7BFBFFFFF77BFBFBFFFFFEB
:10064000FFFFBFBFB75BFFFFBFBFA464FFFFBFAD2E
:10065000A47FFFFFBFA4BF7FFFBFADBFBFBFFFB67B
:10066000BFBFBF77F7BFBFBF7777FFBFBFBF6452C2
:100670006D7F6E2E2D2D7F766E6E6E2E7777777650
:100680002E1C7F776E251C25776525251C096E6E2F
:100690001C0949255B494A6E7F645377BF775B5CD1
:1006A000256E6E255B4A25651C1B5B002524245B9B
:1006B00053001C1B5B5C00000A5B64000000646468
:1006C000000000005C0000000000000000000000CE
:1006D0005B5C7FBF77765C6D7FB777775C6D7FBF44
:1006E00077775C64BFBFBFBF0A5C6EBFBFBF0065EA
:1006F000646DBFBF00005B6D646D00000000125BA5
:100700007777777F6E6E77777F766D7677BF776D49
:100710006E76BF7F6D6E767FBF7676BFBF76BFBFCA
:10072000BFB664ADADB6B6ADBFFF646DADB6AD647A
:1007300077BFBFBFFFFF77BFBFBFFFFF7FBFBFBF99
:10074000FFF6BFB7ADF6FFFFA4ADFFFFFFFFFFFF52
:10075000FFFFFFFFFFFFFFF6A4005B520000000059
:10076000BFBFAD5B64BFB6ADADBFFFBFFFFFFFFF57
:10077000BF64FFFFBFB6765BFFBFBF5B0000FF5CDF
:100780000000000000000000000000000000000069
:10079000BFBF645C5C006E5C654900006D5B00007F
:1007A0000000000000000000000000000000000049
:1007B0000000000000000000000000000000000039
:1007C0000600040000000100020003000400050010
:1007D00006000700080009000A000B000C000D00CD
:1007E0000E000F0010000000110012001300140092
:1007F000150016000600030000001700180019007D
:100800001A001B001C001D001E001F0020002100FC
:10081000220023002400250026000000000208001A
:10082000085504085A0000F8000990000A1E320515
:100830000000FF0000001C0800000000CE45DC4561
:10084000BA46414A2D4ADF45EE45FD45154A0B465D
:100850001946000000010002000300040005010029
:10086000010101020103010401050200020102026B
:10087000020302040205030003010302030303044D
:100880000305040004010402040304040405050034
:10089000050105020503050405050600060106021B
:1008A00006030604060507000701070207030704FD
:1008B00007050800080108020803080408050900E4
:1008C000090109020903090409050A000A010A02CB
:1008D0000A030A040A050B000B010B020B030B04AD
:1008E0000B050C000C010C020C030C040C050D0094
:1008F0000D010D020D030D040D050E000E010E027B
:100900000E030E040E050F000F010F020F030F045C
:100910000F05100010011002100310041005110043
:10092000110111021103110411051200120112022A
:10093000120312041205130013011302130313040C
:1009400013051400140114021403140414051500F3
:1009500015011502150315041505160016011602DA
:1009600016031604160517001701170217031704BC
:1009700017051800180118021803180418051900A3
:10098000190119021903190419051A001A011A028A
:100990001A031A041A051B001B011B021B031B046C
:1009A0001B051C001C011C021C031C041C051D0053
:1009B0001D011D021D031D041D051E001E011E023A
:1009C0001E031E041E051F001F011F021F031F041C
:1009D0001F050505030405060708090A0B0C0D0E83
:1009E0000F10111213141516000000000016051741
:1009F000171717171718191A171717171717171781
:100A000017171717171B1C1D1E1F20212223242513
:100A1000262728292A2B2C2D2E2F00303132333433
:100A200035363738393A3B3C3D3E3F4041424344FE
:100A30000045464748494A4B4C4D4E4F5051525342
:100A4000545556575859005A5A5B5C5D5A5A5A5A6F
:100A50005A5A5A5A5A5A5A5A5A5A5A5A5A010517E7
:100A60000000005A0000000000000000000000002C
:100A70000000000000000000000000000000000076
:100A80000000000000000000000000000000000066
:100A90000000000000000000000000000000000056
:100AA0000000000000000000000000000000000046
:100AB0000000000000000000000000000000000036
:100AC00000000000000000000800000000084800CE
:100AD00000000048084800000008480800000048DE
:100AE00050080000405008500000404050080000EE
:100AF0004000480800000000000000000000000066
:100B00000000000000000000000000005040000055
:100B100000004840000000504040400000085040A5
:100B200040005050000000000000000000000000E5
:100B300000000000000000000000000000000000B5
:100B4000000000000000000048000000000010004D
:100B50000000000000000000000000000000000095
:100B6000000000005000000000005050000000088D
:100B70005050000000505059000050505950000093
:100B8000505950400000000000000000000000002C
:100B90000000000000000000404000000040404015
:100BA0000000404000404000404040814000404044
:100BB0004040400000000000000000000000000075
:100BC0000000500000000000500000000050505095
:100BD000000000505010004050405050508159814A
:100BE00059595940000040505050000040505008A2
:100BF000000040085050004040501050004040500D
:100C00005050008140595008404050505050404092
:100C100059595050500040505050484040400848AA
:100C20004040405050084040505050505040000804
:100C3000505008404050505050504059595050501A
:100C4000404859590000000000000000000000006A
:100C5000500000000000500000000000590000009B
:100C6000000050000000000059000000000050008B
:100C70000000000000000000000000000000000074
:100C80000000000000000000000000000000000064
:100C900000000000000000500000000000500000B4
:100CA00000000050000000000000000000000000F4
:100CB0000000000000000000000000000000000034
:100CC000000000000000000059000000000050007B
:100CD0000000000000000000000000000000000014
:100CE0000000000000000000000000000000000004
:100CF0000000000000000050000000000050000054
:100D000000000850480000000000085000000000EB
:100D100050504000000000504000000040404000A3
:100D20000000404081000000404040000000404082
:100D30004000000000000000000000000000000073
:100D400000000000000000000000000000000000A3
:100D50000000000000000000000000000000810012
:100D60000059599900000000000000000000000038
:100D70000000000000000000590000000050595918
:100D800000590059995959995959599959595959C5
:100D9000A159995900005059504000505959505983
:100DA00000595059505950595950595959598199C8
:100DB00059815981595059409959595959995959F5
:100DC0005981594881814040404040004040404066
:100DD000814040408181408181404040814040814C
:100DE0008140408181815981814081595981814867
:100DF0004859814800000000000000000000000089
:100E000000000000000000000000000000000000E2
:100E100000004000000000008100000000004800C9
:100E20000000000000000000590000000059505070
:100E3000000000595050000059505940005959596C
:100E40005981005999599959599959598140595974
:100E500059814881000000000000000000000000EF
:100E600000000000000081000000000040000000C1
:100E700000008100000000004000000000004881E8
:100E800000484000000000000000000000000000DA
:100E9000000000000081000000000081008181004E
:100EA00040814040818181814040594048404059C3
:100EB0005981815950595059508150595050404092
:100EC0008159595940815959995059408148595926
:100ED00059818159595050005050594850595959C9
:100EE000995959594040000000004081000000001D
:100EF00040400000000081404000008159408100D6
:100F00004040505081818181995959404081619977
:100F100059814881814040505059408181505950F9
:100F200040405059595981815999595040408159EF
:100F30009959814040595959814081595999484896
:100F400050995959405950595950815959595981B5
:100F5000818159505040504050598181598159994F
:100F600040405981595981595959595981594050CD
:100F7000509940595000000000005000000000004F
:100F800059000000000059005900000050005000B6
:100F90000000A1005059590059595050500059595A
:100FA0005999595900000000505900000000505054
:100FB0000000000059500000005059590000005036
:100FC0005959000000599959000000505959000022
:100FD00000595959500050500000595050590000C4
:100FE000505050500050594059595040508159501C
:100FF0005981595959595059509981A15959A15953
:101000004850995900000000000000000000000056
:1010100000000000000000000000000000000000D0
:101020000000000000000000000000590000000067
:101030005059590000000000505000000050505915
:101040000000005059500000005059500000505905
:10105000595900005950595000505959505959592F
:1010600059815959404040400000404040400000F4
:10107000504081400000994040815000598181409A
:10108000590059505081408159595959404050A1F7
:1010900059814081595059505959996159995089EC
:1010A0005950506189898959D289898961A1618999
:1010B000895999A1998961A1595950595959A150F2
:1010C00059A1595050005959615040898950599936
:1010D0004889895959A18A898989A1598989495990
:1010E00059A189895959A1595989A1A159A1A15930
:1010F0008969A161599959898189595959508989B1
:101100005999595959895959505949895059898971
:101110008989A159A159898950A159895059695979
:10112000898961A148895089898189894848898943
:1011300089498989894889898A8949898A898A89DD
:101140008989595948898959A1A15989895961A120
:10115000A189A1A1898189000000898989000000F5
:1011600089898989000089894948000050898A89CC
:101170008900595989D28900A1A15989810069A1A1
:1011800059598989000000000059000000000059E9
:101190000000005900590000A1A1A1A10000595967
:1011A000A15900009959595000A161A159A100A16C
:1011B00059A161A1995989488189A1598989898948
:1011C00059995950488959595948898959A1994972
:1011D000895099594889595959895999595989A111
:1011E000595999A189890040890089810049488914
:1011F00089890089898989894989898A59494989D7
:101200008989898959598989488959A18959995957
:10121000595989590000000000000000000000003A
:101220000000000000000000000000005900000065
:101230000000A18900000000A18900000000598978
:10124000000000000000000000000000000000009E
:1012500000000000005900000059A159000000A141
:1012600059A10000599961990000595999610000EC
:1012700059A161995959A159895959995959598966
:1012800099599959A159A161A1595959599961A1DE
:1012900099595989A1A159A1A1898989485989894F
:1012A0008989488950A15959599959595959995970
:1012B0009959A1595959A15959595959598959A156
:1012C0005959A189A159595959A159A148898959EF
:1012D000996199595950598959895959595999595F
:1012E00059595959595959599959599959595959EE
:1012F00059895959995989488159A159898961A1AF
:1013000059508959590000000000814889000000A7
:1013100089898900000059894859000089618999A3
:1013200000005989A15900005048A1590000A19915
:101330005959000000000000004800000059598978
:1013400000595999598900A159595048005999593A
:10135000A1895959A161A15959A159505059A1596F
:10136000A15961A18959595959994859995999616E
:10137000505959A161999959A1A1595959A159593E
:1013800059A18959A1A1A159A1595959A15959A1A5
:1013900059A159A189A1595959998959A15959A1B5
:1013A00059A1599959595959595959999959A1A115
:1013B00061A161A159A1594099A1A161898959618E
:1013C00059A199895999A1615999A159599959A135
:1013D00059A15959A159598999A1A159898989892D
:1013E00050A1898989898959894989D289898989B5
:1013F0005981994800000000000000000000000032
:1014000059A100000000A1590000000059A10000EE
:101410000000A161000000008999A15900009961B4
:10142000A1590000000000000000000000000000C2
:1014300000000000000000000000000000000000AC
:10144000000000000000008900000000008900008A
:1014500000000089000059590000000099615900FE
:10146000000059995950595999599959A199615957
:1014700059A1485959A1A159599959A161A1A161ED
:10148000A159995900000000000000000000000070
:101490005989000000009989000000008959000066
:1014A000000059A10000000059590000000059A196
:1014B00089000000000059509959005959A1595903
:1014C00000990850995000595959615959599959D9
:1014D00099595999A1598961995961A189A161992C
:1014E000599959A1A1599959595999595959596114
:1014F0005959595959A159995948595999595959A5
:101500009959A1599959A15959A16199595989894B
:1015100061A1618159000000000059000000000035
:10152000A10000000000590000000000A189000097
:101530000000894800000000485900000000599947
:10154000000000000000000000000000000000009B
:10155000000000000000000000000000000000008B
:10156000000000000000000000000000000000007B
:101570000059598900000000000000000000000030
:1015800000590000595900A159595059A159599968
:10159000595008595059A189505999898989A1A14F
:1015A00061A1898900005959995900599959595986
:1015B000995959A1995959500059596181488989B6
:1015C0005099894889895959998989898959598AA4
:1015D0008948599999598159505959599959509946
:1015E00099595959895950599959408959595959AD
:1015F0005989A15999599950595950505989A15906
:101600005989488959595981818159A181894861EC
:101610005948484899595959995959895999615975
:1016200089A1A1615059596159995999A159A1614B
:10163000A16159A15059995959A1A1A1A1995999AB
:101640005959A159A159A1A159A15999A1A1A1A142
:10165000A1A1A1A1A1A15999A1A1A1A1A1A1A1A1CA
:10166000A1A1A1A14859A1995950A199A1594808EE
:101670005959995959A159A159A1A159A1A1A1A15A
:10168000598999A1A1A1A189A19959A1A148A1A173
:10169000A1A189A19989A159995959485959A1A13B
:1016A00089A1A1A1A159995959A1A1A19959A1A172
:1016B000A199A1A1A1A1A1A1A1A1A1A1A1A1A1A122
:1016C000A1A1A1A1A1A1A1995959A1A199A1A159F2
:1016D00099A1A159A1A1A159A15959A1A150A159BB
:1016E000A15959A159A1A1A1A1A1A1A19959A1A112
:1016F00059A1A1A15999A1A1A18999A1A1A1A189AA
:10170000A1A159A1A1A1A1A1A159A159A1A1A1A1A1
:10171000A1A1A159A1A1A1A159A1A1A1A1A1A1A149
:10172000A1A1A1A1A159A1A1A15989A1A1595999E9
:10173000A1899959A1A1995989A159A1A1A1A159F9
:10174000A1A1A1A1A1A9A1A1A1A1A1A159A1A1A1C9
:10175000A1A1A1A1A15959996959A19959A1595971
:101760005959A1A199A1995959A159A1A1A1A15929
:1017700059A1A1A18989A1A1A159A1A1A159A1A161
:10178000A1A1A159595999898969A1A18999A199B9
:10179000A1A1A15959A1A1895950595959895999BA
:1017A00059A189A1A1A1595948A1A1A1A1A148A1CB
:1017B00059A1A1A1998989000000A189890000008F
:1017C000A1A18900008959A18A00008959995189EC
:1017D0008A99995989898989A1A159898959A19990
:1017E000898989A148A1A161995989A15999A1899A
:1017F000A15959A1A189A1995959508A99A1A189A1
:101800008959A1A15959A1A1995999A1A1A1A1A110
:10181000A1A1A1A189D2484048898989998989993A
:101820008989598989A18959A159999989A1A1A120
:101830008959A1A1A1595989A1A159A1A159A1A130
:10184000A1A1A1A189A161A159A18950A159A15921
:10185000A15959A1A199A1A1A159A1A19959A199B0
:10186000A1A1A1A150A1A1A189A1A199A1A1A189F1
:10187000A1A1A1595959A18989A159A18999595958
:10188000A159595059A1A1995959A15999A1A1A159
:10189000A159A15959A1A1A1A1A1A1A1A1A1A1A110
:1018A000A1A1A1A15961A15900A19961995900591A
:1018B000595959A1A1A159A1A1A1A159A1A1A159C8
:1018C0005959A1A15999A1A199A1A1A159A1A1A138
:1018D000A1A1A1A1A1A15959A19961A1A1595959A8
:1018E000A1A1A1A1A1A1A1A1A1A1A1A1A1A1A1A1E8
:1018F000A1A1A1A1A1A1A1A1A1A1A1A1A1A1A1A1D8
:10190000A1A1A1A161898989A1599959598959A18F
:101910006159995989595959A1A169D2A1A159501F
:101920005000A1A1A15959A1A1A1A159A159A1A1B9
:10193000A1A1A1A1596199595989A1A159595999AF
:10194000619961A1A161A1619950A15989A15961D0
:10195000A1A189A1A1A1A161A148A1A1A1A1A1A128
:1019600089A1A1A18989A1A1596140505961A1A171
:1019700089899959595949899959A1A1A18959998F
:1019800059A1D28999A1619961D2894899A1A15996
:101990008989A1A1A161A1A1000059A1616159A1F9
:1019A0005999A1A1A1085959A15961A161A159A1B0
:1019B00050A159A16159A161A15999A1A1A1A1A1C8
:1019C000A1A1A1A10000008989890000008989994D
:1019D000000089A159898A898961A1508989619901
:1019E000A161A189A16161A161A169A1A159A1A17F
:1019F000599959A159A1A1A1590859A15961A1A168
:101A00005959A199594889A1596189A1A159A18917
:101A1000A159A1A1A9A1A1A1A1A1A1A1A18959A156
:101A2000A15989A1998989000000504889000000C6
:101A30008989890000005948899A8A8AA159898A26
:101A4000D29A5999A1898989A1A14889898AA1999C
:101A5000894989890000000000A1000000008AA1D6
:101A60000000008A89590000005189A10000008906
:101A700089598900598951A189A1894940594889C1
:101A8000894889A1A159A161A1A161A1A159A15927
:101A90009961A159A1A1619959D25959A16959894D
:101AA000A159A199598989A159A1A189A1A1A1A14E
:101AB0005989A1A189A19961996189A161A159A1BE
:101AC000898959A159A15961A159A16150A1A1A127
:101AD000A199A1A1A1A1A159A1A1A1A1A1A1A1A146
:101AE000A1A1A1A1A159610000005959A1898900B2
:101AF000599959898A00A159A18A8A0059A148890E
:101B0000A100A1A1484859595989898959A189A198
:101B1000A1A1A15900000000000000000000000089
:101B200000000000000000000000000000000000B5
:101B30000000A1000000008AA15959000089A1A15C
:101B4000A1A1A1A10000895059A10000595999599A
:101B50004800A1A161A18989A15908485189595911
:101B600050598A8AA1A1A1A189A1A159595989597C
:101B700099A189A15961A1598961A159595059590E
:101B800059A15059A1590850A159995959A1A1A138
:101B900059A1599959A1A1A1A1A1A1A1A1A1A1A115
:101BA000A1A1A1A15989895999A1995989A1A1A155
:101BB00050A159A1A1A1A1A1A1A1A159A1A1A1A1F6
:101BC000A1A1A1A1A1A1A159A1A1A1A1A1A1A1A14D
:101BD000A1A159A1A1A159A15989A1A1A159895096
:101BE000A1A1598989A150598959A159089989599F
:101BF00059A1A189A1A1A1A15999A1A1A1A18959E5
:101C0000A1A1A1A1A1A159484808A1A1A15959592F
:101C1000A1A1A1A1A159A1A1A1A1A1A1A1A1A1A1FC
:101C2000A1A1A1A1A1A1A1A1A1A1A1A1A1A1A1A1A4
:101C3000A1A1A1A1A1A1A1A1A1A1A1A1A1A1A1A194
:101C4000A1A1A1A1A1A1A1A1A1A1A1A1A1A1A1A184
:101C5000A1A1A1A1A1A1A1A1A1A1A1A1A1A1A1A174
:101C6000A1A1A1A1A1A1A1A1A1A189A9A1A1A1A174
:101C7000A1A1A1A1A1A1A1A1A1A1A1A1A1A1A1A154
:101C8000A1A1A1A1A1A1A1A1A1A1A1A1A1A1A1A144
:101C9000A1A1A1A1A1A1A1A148A1A1A1A189484857
:101CA000A1A1A1A1A189A1A1A1595948A1A1A1A125
:101CB000A1A1A1A1A1A1A1A1A1A1A1A1A1A1A1A114
:101CC000A1A1A1A1A1A1A1A1A1A1A1A1A1A1A1A104
:101CD00089A1A1A1A1A189A1A1A1A1A15989A1A184
:101CE000A1A1A1A1A1A1A1A1A1A150A1A1A1A1A135
:101CF000A1A1A1A1A159A1A159A1A9A148A1A1A1B5
:101D0000A1A189A1A1A1A1A1A989A1A1A1A1A1A1EB
:101D1000A1A1A1A1A1A1A1A1A1A1A1A1A1A1A1A1B3
:101D2000A1A1A1A1A1A1A1A1A1A1A1A1A159A1A1EB
:101D3000A1A1A1A1A1A1A1A1A1A1A1A1A1A1A1A193
:101D4000A1A1A1A1A1A1A1A1A1A1A1A1A1A1A1A183
:101D5000A1A1A1A1A1A1A14889A1A1A1A1A189A1FC
:101D6000A1A1A1A18989A1A1A1A1A189A1A1A1A1AB
:101D7000A1A1A1A1A1A1A1A1A1A1A1A1A1A1A1A153
:101D8000A1A1A1A1A1A1A1A1A1A1A1A1A159A159D3
:101D9000A1A1A1A1A1A1A1A1A1A1A1A1A1A1A1A133
:101DA000A1A1A1A1A1A1A1A1A1A1A1A1A1A1A1A123
:101DB000A1A1A1A159A1A1A1A1A1A159A1A1A1A1A3
:101DC000A1A1A1A1A1A1A1A1A1A1A1A1A1A1A1A103
:101DD000A1A1A1A1A1A1A1A1A1A1A1A1A1A1A1A1F3
:101DE000A1A1A1A1A1A159A1A159A1A1A1A159A1BB
:101DF000A1A1A1A1A1A1A1A1A1A1A1A1A1A1A1A1D3
:101E0000A1A1A1A1A1A1A1A1A1A1A1A1A1A1A1A1C2
:101E1000A1A1A1A1A148898949408989A189A14895
:101E2000A1A1A18999A1A15999595959A1A1A1A1EA
:101E3000A189A1A1A1A199A1A1A1A1A1A1A1A1A1B2
:101E4000A1A1A1A14948898989A14889A189A1A104
:101E50008989A1A1A1A189A1A1A1A9A140A1A1A113
:101E6000A1A1A1A1A1A1A1A1A1A1A1A1A1A1A1A162
:101E7000A1A1A1995948898948A1A9898989A1A1C4
:101E8000A14848A1A1A1A1898989A1A1898989899C
:101E9000A1A189898989A1A199A1509999A150A14C
:101EA0009999A1A1A159A1A1A1A1A1A1A1A189A192
:101EB000A1A1A189A1A1A1A989A1A1A1A1A1A1A13A
:101EC000A1A1A1A1A1A1A1A1A1A1A1A1A1A1A1A102
:101ED000A1A1A1A18959A1A1A1A1A189A1A1A1A16A
:101EE000A1A1A1A1A1A1A1A1A1A1A1A1A1A1A1A1E2
:101EF000A1A1A1A1A1A1A1A1A1A1A1A1A1A1A1A1D2
:101F0000A1A1A1A1A1A1A1A1A1A1A1A1A1A1A1A1C1
:101F1000A1A1A1A1A1A1A1A1A1A16939A1292939A9
:101F200079797979797979393979397979797979E1
:101F300079797979A1A1A1A1A1A1A1A1A1A1A1A131
:101F4000A1A1A1A1A1A1A1A1A1A16939A129293979
:101F500079797979797979393979397979797979B1
:101F600079797979A1A1A1A1A139A1A1A169393971
:101F70006969397979393939397979797939797971
:101F800029797979797979397979793979397979D1
:101F900079397918797969793979697979397979F2
:101FA00039793979292139797921292939796918B2
:101FB00069397939297939797929793979392169E9
:101FC0003979792929212979697939697929392949
:101FD0007939792979796939797979296939793931
:101FE00029793969397979396939397979397929A1
:101FF0007929693939297929396979793979212111
:1020000039397939692979397939792939793979B0
:102010003979793969397939693979397939797910
:1020200039796939393929211821212921212118A2
:102030006921212118217969296121213979796959
:10204000212179792939182179797929391879293A
:1020500039211818A1A1A1A1A1A11818A1A1A1A17C
:1020600021211821A1A1182121211861182129213C
:10207000212118292121212921182129212121214A
:1020800029212121A1A1A1A1A1A1A1A1A1A1A1A138
:10209000A1A1A1A1A1A1A1A1A1A1A1A121A1A1A1B0
:1020A000A1A1216161A1A1A121292121A1A1212118
:1020B00029292121A1A1A1A1A1A1A1A1A1A1A1A100
:1020C000A1A1A1A1A1A1A1A1A1A1A1A1A1A1A1A100
:1020D000A1A1A1A1A1A1A1A1A1A1A1A1A1A1A1A1F0
:1020E000A1A1A1A1A1A1A1A1A1A1A1A1A1A1A1A1E0
:1020F000A1A1A1A1A1A1A1A1A1A1A1A1A1A1A1A1D0
:10210000A129A1A1A1A12979A1A1A1693969A1A1AF
:10211000A1396939A1A1A1A1A1A1A1A1A1A1A1A1B7
:10212000A1A1A1A1A1A129A1A1A1A1A17929A1A1B7
:10213000A1A1297979292169396929397939793927
:10214000797939797979797979797979797979793F
:1021500079797979797979797979797979797979EF
:1021600079797979797979797979797979797979DF
:102170007979392179792979297979797939792997
:10218000797929693979792979397979397939697F
:1021900079793979297979797929797979792979DF
:1021A000397979793979297939797929793979397F
:1021B000297929793979797979797979797979796F
:1021C000397979797979793979797979397979793F
:1021D000797979392979297939797939792979296F
:1021E000297979397939397939793979397939697F
:1021F0002979792979397921397979292121792917
:1022000021212179393979393969797939797939D6
:1022100079397979292139693918212139792121A7
:102220001821212118212121212129212121397938
:102230003979212139792118182169211818211893
:102240002118212121212129211821292118212189
:1022500021212121212121212121212121217969CE
:1022600021217969182921212129212121212921AF
:102270002121292921212929212121212921292916
:102280007979212979393979796939797939392906
:10229000797939792121212121292121211821210F
:1022A0002921212121186939792121213979397987
:1022B0002921397929792129793979212121297906
:1022C000212121212929A1A1A1A12121212121A16E
:1022D00021212121212121212921292121212121DE
:1022E00018212118212121212121212921211821F1
:1022F00021212121A1A1A1A1A1A1A1A1A1A1A1A1CE
:10230000A1A1A1A1A1A1292121A1A1A12121212135
:1023100021A1292121211821212121212121212926
:1023200021217939A1A1A1A1A1A1A1A1A1A1A1A12D
:10233000A1A1A1A1A1A1A1A1A1A1A1A1A1A1A1A18D
:10234000A1A121A1A1A1A1A1212121A1A1A1792125
:10235000292118A1A1A1A1A1A1A1A1A1A1A1A1A1EE
:10236000A1A1A1A1A1A1A1A1A1A1A1A1A1A1A1A15D
:10237000A1A1A1A1A1A1A129A1A1A1393979A12935
:1023800079397979A1A1A1A1A1A1A1A1A12121A11D
:10239000A1A121211821A13939792121397969395E
:1023A00079397929792979693979397929393979DD
:1023B00039693979A1A1A1A1A1A1A1A1A1A1A121BD
:1023C000A1A121182929212129292179212921297E
:1023D0007939392129397979791869793939793906
:1023E00079293979A1A1A1A1A1A121A1A1A1A1A18D
:1023F0002121A1A1A1A1212121A1A1A13921212135
:1024000021A17939792921213979397929217979D4
:1024100029792918A1A1A1A1A1A1A1A1A1A1A1A14D
:10242000A1A1A1A1A1A1A1A1A1A1A1A1A1A1A1A19C
:10243000A1A1A1A1A1A1A1A121A1A1A1A1A121210C
:1024400018A1A1A1A1A1A1A1A1A1A1A1A1A1A1A105
:10245000A1A1A1A1A1A1A1A1A1A1A179A1A1A1A194
:102460002939A1A1A1297979A1A139793939A1798C
:1024700039797921A1A139793921A139693921180D
:1024800079793969217939397929793969792179DC
:1024900039792921297929792121793979292169DC
:1024A000297939796979393979293979797939798C
:1024B000792939397979793979797979397939395C
:1024C000797939797979397979393939793939694C
:1024D00079793979797979292129796921217939A4
:1024E000292118793979181879397979217939793F
:1024F000797979797979797979797979797979794C
:10250000797979797979797979797979797979793B
:10251000797979797979797979797979797979792B
:10252000797979797979797979797979797979791B
:102530007979797979797979292179797939796903
:10254000797979397939796939793969793979399B
:10255000793979793979296979797929793979795B
:102560003979397921397939792979397929793953
:10257000397939793979792979297979792979797B
:1025800079793979797979797979797979797979FB
:1025900079797979793979397939797939793979EB
:1025A000392979297979797979797979797979797B
:1025B000797979797979797979797979797979798B
:1025C000797979797929793979392979397929792B
:1025D00079797979792979797979797979797979BB
:1025E000792979797979793979797979297979397B
:1025F00079297939797929397939397979291821F4
:1026000079391821397939793969793979396939D3
:10261000792979693979397929397929793979792A
:1026200029793979212118182179212121793939FC
:1026300079397939797979397929792979297939FA
:1026400069393979397939797939693979397979DA
:102650007979797979216979212179393929791833
:1026600029697979397939793939396969397979DA
:1026700079297939792979392979397939797939FA
:10268000793979292921792979396939693979217A
:1026900039693979397939792979297979297939EA
:1026A0007939793979791821297939292121291814
:1026B0002169397929292121212121292921212132
:1026C0003979211829212121212121212121217933
:1026D000397929793979397979297939792939799A
:1026E000297939792121A1A1A139211821397969C3
:1026F00021793979393979297929696939793979A2
:102700003979297979297939792939793979693979
:1027100069793979397939793939397939797979F9
:102720007939693929393969397979797939792959
:1027300029793979397979217929792121393979B1
:102740003979397979396939793929793979396929
:1027500079297939792139793979397979397979D1
:102760003979217939793979793979297929693921
:102770007939792929793979693979212139796939
:102780002129797939292979393969793969797921
:1027900029216939392121217939697939697939C9
:1027A00079396939397939792121397939212121E1
:1027B00079212121212139212921792921212179D9
:1027C00039792169397929793979397939797939B1
:1027D000792979212121212118A1212921212121B2
:1027E00079297921212179396939212139693921D9
:1027F0002129392121212121212121292129212199
:1028000021212121A1A1A1A1A1A1A1A1A1A1A1A1B8
:102810002121A1A1A1A121212121A1A121211821B1
:10282000A1A121212129A1A1292918212121292181
:1028300029182121A1A1A1A1A1A1A1A1A1A1A1A189
:10284000A1A1A1A1A1A1A1A1A1A1A1A1A1A1A1A178
:10285000A1A1A1A1A1A1A1A1A1A1A1A1A1A1212168
:10286000A1A1A1A1A1A1A1A1A1A1A1A1A1A1A1A158
:10287000A1A1A1A1A1A1A1A1A1A1A1A1A1A1A1A148
:10288000A1A1A1A1A1A1A1A1A1A1A1A13979A1A1C8
:10289000A1397939A1A1A1A1A1A1A1A1A1A139A188
:1028A000A1A1A1797939A1A139393979A1297979F8
:1028B00079393979392979296939697939797929D8
:1028C00079397939A1A1A1A1A1A1A1A1A1A1292110
:1028D00029A1A12121217929292179217939697910
:1028E0002929793979297921297939792129793958
:1028F00079212121A1A1A1A1A1A1A1A1A1A1A1A170
:1029000021A1A1A1A1A12121A1A1A1A1212921212F
:10291000A1A1212121212121212121211829292998
:1029200029396921A1A1A1A1A1A1A1A1A1A1A1A12F
:10293000A1A1A1A1A1A1A1A1A1A1A1A1A1A1A1A187
:10294000A1A1A1A1A1A1A1A121A1A1A1A1A12121F7
:1029500021A1A1A1A1A1A1A1A1A1A1A1A1A1A1A1E7
:10296000A1A1A1A1A1A1A1A1A1A1A1A1A1A1A1A157
:10297000A1A1A1A1A1A1A129A1A1A1293979A1A1C7
:1029800039797918A1A1A1A1A1A1A1A1A1A1A139E0
:10299000A1A1A1793979A179293939697929797977
:1029A0007939793979297939392129793969217937
:1029B000397939793979392921797939212139795F
:1029C0003969797969393979293939797929796987
:1029D00079397939393979793979797979792979F7
:1029E00079797979397939792979297979397939F7
:1029F0007939297929797939797939693979397937
:102A000039693979793969397979792979397979E6
:102A1000797929792979292139797939792979793E
:102A20003979297939797939793969393979297946
:102A3000392979297929212979212169397939791E
:102A40002979397979797979797979797979797986
:102A50007979797979397979797939797979797966
:102A600069797979797979797979797979797979E6
:102A700079797979796939796979793979397979A6
:102A80006979397979797939797979797979797946
:102A900079797979797979797979797979797979A6
:102AA0007979797979797979797979797979797996
:102AB0007979797979297979797939797979297966
:102AC0006939796979397969797979797979797926
:102AD0007979797939796939797979297979397986
:102AE00039793939693979797979797979297939F6
:102AF0007939397939792979797979797979797956
:102B00007979797939697929797939397979797955
:102B10007979797979797939797979797979797965
:102B20007979797979797979797979797979797915
:102B30007979797979793921217939697979396995
:102B40007939693979393979397939797979797985
:102B50006939797979793979797979797979797975
:102B60007979797939792979793979397929792985
:102B700069793979397979397939797979797969E5
:102B80007939397939793979796939797939797945
:102B900079792979792979212139792921212121E5
:102BA00079792121212129397921297979212179DD
:102BB00079396979397939797929797979397979E5
:102BC0007929797939792939693918797979397986
:102BD0003979397979397979212118797939797976
:102BE0007979697979797979797979797979797965
:102BF000797979792921693979797979797979793D
:102C00007979797979797979797979797979797934
:102C10007979797979797979797979797979797924
:102C200079797979797979792979797979797939A4
:102C300079797929397979797979797979797939D4
:102C40007939793969793969397979297979796974
:102C5000397921183979297939697979397979393D
:102C600069397969397939797939792179397921E4
:102C700018217979212121212118292129792179E6
:102C80007979792979793969212129797921212954
:102C900079182129212121212121212121212121CD
:102CA000212118212129212179791821797979394E
:102CB00079693979212921212129212121212118ED
:102CC000212121212121212121212921217979213C
:102CD000217979397979793979793979396929791C
:102CE00069397979212121212121212121212121C4
:102CF00021211829212179792921212179397979ED
:102D0000212179793979792179396979397939794B
:102D100079297979212121A1A1A121212121A1A113
:102D20002121292121212121212921212121212183
:102D300021292179211821297939797921212979A4
:102D400079397979A1A1A1A1A1A1A1A1A1A1A1A153
:102D5000A1A1A1A1A1A1212129A1A1A121212121DB
:102D600029212129212118212121212121297921EC
:102D700021212121A1A1A1A1A1A1A1A1A1A1A1A143
:102D8000A1A1A1A1A1A1A1A1A17979392139793963
:102D900069792121217939392118182118792121BE
:102DA00021212121A1A1A1A1A1A1A1A1A1A1A1A113
:102DB000393979A13929797939297979792979794B
:102DC0002979797929792979397979797969187914
:102DD00039693979A12939693979A1797939792913
:102DE00039793979793979396979797939797979A3
:102DF0007979792979797979397939797979792963
:102E000069797979297939793979793979396921FA
:102E10007969396939797979797979797979693912
:102E200029797979797979397979797979797979A2
:102E3000797979792979392121212121212129794A
:102E40007921217929793979397979392979796912
:102E50003979797939797979397979397929793972
:102E600079693979792179793969397939397939CA
:102E70002979797939217979392118793979297933
:102E800079796929797979797979793979297979A2
:102E9000397969793979212921A17921212121796A
:102EA0001879397939797939697979393979793983
:102EB00069797979397939697939797979393979E2
:102EC0006979797929797939297979397969792902
:102ED00029793979397979397939797979797979B2
:102EE00039693939793979397979297979797979F2
:102EF00079797979297969397939793979397979A2
:102F000039793979793979796979397939397979C1
:102F10007979797979797979797979797979797921
:102F20007979797979797979793979797979797951
:102F30007979797979797979797979797979797901
:102F400079797979797979797979797979797979F1
:102F50007979797969397929793979793979797901
:102F60007939797979793979697979797979797961
:102F70007979797939797979797979797979797901
:102F80007979797979797929797979797979797901
:102F900079797979797979797979797979797979A1
:102FA0007979797979797979797979797979797991
:102FB00079797979397979797979797979797979C1
:102FC0007979797979797979797979797979797971
:102FD0007979797979797979797979797979797961
:102FE0007979797979797979797979797979397991
:102FF00079797979693979797929797979797979E1
:103000007979797979797979797979797979797930
:1030100079797979297921217979797969397939B0
:1030200069397979697979797979397979797979B0
:103030007979797979797979797979797979797900
:1030400079797979792979397979797979793979C0
:1030500039792979697969797979793979797979D0
:1030600079797979797979797979797979797979D0
:1030700079797979797939797979297979397939D0
:103080007939797979697979797979797979797900
:1030900079797979797979797979797979797979A0
:1030A0007979797979397979793979797929797960
:1030B0007939797969397979797939797979797950
:1030C0007969797979797979797979797979797980
:1030D0007979797979793979792979797929797940
:1030E0007929797979297979792979793979797980
:1030F0007939797979797979797979797979797980
:10310000797979797979396979397979793979690F
:1031100079396979792179692121212121217969F7
:10312000797979693979797979797979797979795F
:1031300079797979797969212121391821212179C0
:1031400021212169797969797979792979397979A7
:1031500079797979797979797979797979797979DF
:1031600079797979217921211821797979797921E8
:1031700039693969396979797979797979797979AF
:1031800079797979797979797979797979797979AF
:103190007979797921182121217921797969392160
:1031A000796939797979792979797939797979796F
:1031B000797979797979797979797979797979797F
:1031C0007979797939797939797921797969797957
:1031D000792121792979797979397979797979799F
:1031E000797979797979797979797979797979794F
:1031F000797979797979797979797979797979793F
:10320000797979797979797979797979797979792E
:1032100079797979797979797979797979791818E0
:103220001818181879797979797979797979797992
:1032300079797979797979797979797979797979FE
:1032400079797979797979797979797979791818B0
:103250001818181821212121212121212121212182
:1032600029292929292929292929292929292929CE
:1032700029292929292929216C2323231B1C231CC3
:103280001C1414542121212121212121212121211A
:10329000292929292929292929292929292929299E
:1032A0002929232B232329291C5B1C1B2323141DC1
:1032B0001C141D64212121212121212121212121D1
:1032C000292929292929292929292929292929296E
:1032D000292929292323232A2323631C1C1B251C7A
:1032E000251D5D542121212121212121212121215F
:1032F000292929292929292929292929292929293E
:1033000029292929292929291A2321292929151C6B
:103310001D241B21212121212121212121212121A4
:10332000292929292929292929292929292929290D
:1033300029292929292323232323231B1C1C1C146B
:103340001414541521212121212121212121212160
:1033500029292929292929292929292929292929DD
:1033600029292323292929295B1B23232B231D14E6
:103370005C1C641C212121212121212121212121C9
:1033800029292929292929292929292929292929AD
:103390002929692163236A6923241C1C1C22255DB9
:1033A0001D15141421212121212121212121212137
:1033B000292929292929292929292929292929297D
:1033C00029292929292929292323292C23231D6453
:1033D00023231C1C212121212121212121212121E3
:1033E000292929292929292929292929292929294D
:1033F00029292929292929216B2323231B1C231C43
:103400001C14145421212121212121212121212198
:10341000292929292929292929292929292929291C
:103420002929692263236B6923241C1C1C22255D26
:103430001D151414212121212121212121212121A6
:1034400029292929292929292929292929292929EC
:1034500029292929292929226C2323231B1C231CE0
:103460001C14145421212121212121212121212138
:1034700029292929292929292929292929292929BC
:10348000292929292323232B2323631C1C1B251CC7
:10349000251D5D54212121212121212121212121AD
:1034A000292929292929292929292929292929298C
:1034B00029292929292929291A2322292929151CB9
:1034C0001D241B221D1C5D1D1D5E5E6767676767EF
:1034D000666F676F666F666766666766666766666D
:1034E0006627155D1D151D5D14155D5D1D151415F3
:1034F0001515551566665E651515676F67661D1DA2
:1035000067661D151414265D1D5D14155D155D158A
:10351000141415141414151D1454151414661415CC
:1035200014141D67555D55155D151514151D1514DD
:103530001415145EAF6F14145D6F6766151D676F09
:1035400067666666676F6766676F6F6767666667F9
:1035500066676766141454145C1515141415141555
:10356000A7671D5D1E5D66665E1D151D1E1D665EE0
:1035700014151E5D151D5D145E155D5D15155E1D32
:1035800015155D1415541414141414155D15151423
:1035900014151D1D655E15151D5E6667155D1566A6
:1035A0006F6F66666667676F676F67666767676F87
:1035B0006727666F151454155D6714151D1D1E666B
:1035C00066665E1E5D156F66665D151527661D15C0
:1035D000155D661E1E1D1D1567665D551515676612
:1035E0001E1D14146766662766261E1E1D1D155DAA
:1035F0005D1D555D1D1515551E1D15151D155D14FB
:103600001414551515541515145D15141414151DA1
:103610005D1514141E5D151414151D1554155D1437
:1036200054151D15155414145C15141D1415151D71
:103630005D145C14141415661514141D66671414B7
:10364000156667676F67676666666766671E1E1E34
:103650006626665D1D5D675E1E1D5D1D1D5D1D553B
:103660001514155D1514141D151415145D66000050
:1036700000000000665E141515675E1D151D666668
:103680001D5D1D5E676F151566676F67155D666664
:1036900066665D1E1E5E1E666F5D1D141E150000B3
:1036A000000000006F6F6666665D6767671E1554F1
:1036B0006F6F661D141567665D15141466661E1D12
:1036C00054151E5E15151D145D1D5414155D000066
:1036D00000000000155D67676F6614156666672752
:1036E000141D6666266654151D1E666614145D1E3E
:1036F0001D1E1515155D1D545C14141515140000C0
:10370000000000002005010101010101010101018A
:103710000101010101010101010101010101010199
:1037200001010101010102030405060708090A035A
:10373000040506070B090C030D0E06070B090C0305
:103740000D0E06070B090F1011120F1011120F109A
:1037500011120F1011120F1011120F1011120F1061
:1037600011120F1011121314151613141516131429
:103770001516131415161314151613141516131401
:103780001516131415161718191A1718191A1718C9
:10379000191A1718191A1718191A1718191A1718A1
:1037A000191A1718191A200501020304050607083B
:1037B0000909090909090909090909090909090979
:1037C0000909090909090A0B0C0D0E0F1011121332
:1037D000141516091718191A1B09090909090909E5
:1037E00009090909091C1D1E1F2021222324252641
:1037F0002728292A2B2C2D2E2F3031090909323365
:103800003435363738393A3B203C3D203E3F402066
:103810004142434445464748494A4B4C4D4E4F5020
:10382000515253545520565720202020202020202C
:10383000205859205A5B5C5D5E5F60616263642062
:103840005920202020202020200601010101010113
:103850000101010101010101010203010101010155
:10386000010101010101010101040101050601013C
:1038700001010101010701010108090A010101011A
:10388000010B0C01010101010D0E0F1011121301AA
:10389000141501011617180101191A1B0101010164
:1038A000011C1D010101011E1F20212223242526A8
:1038B0002728292A2B2C2D2E2F3031323334353620
:1038C00001373839013A3B3C3D3E3F404142434499
:1038D00045464748494A4B4C4D4E4F505152535420
:1038E00055565758595A5B5C5D5E5F5F5F5F5F5F1F
:1038F0005F6061625F635F5F5F5F646566676869A1
:103900006A6B5F5F6C5F5F5F6D5F160400010203AF
:103910000405060708090A0B0C0D0E0F0E100E11F8
:10392000111111111111111111111213131313137C
:10393000131313141315161718191A171B1C1D1E11
:10394000121F2021222323231324131111111111DB
:103950001111111111112526272627262726272682
:1039600027111111FEFEFEFEFEFEFEFEFEFEFEFE15
:10397000FEFEFEFEFEFEFEFEFEFEFEFEFEFEFEFE67
:10398000FEFEFEFEFEFEFEFEFEFEFEFEFEFEFEFE57
:10399000FEFEFEFEFEFEFEFEFEFEFEFEFEFEFEFE47
:1039A000FEFEFEFEFEFEFEFEFEFE85FEFEFEFEFEB0
:1039B000C6FEFEFEFEFEC7FEFEFEFE00C700FEFEC9
:1039C000FE00C700FEFEFEFE00C7FEFEFEFEFEC7B6
:1039D000FEFEFEFE00C7FEFEFEFE00C7FEFEFE006F
:1039E00000C7FEFE85C60000FE85C6C7C7C785C6E0
:1039F000C7C7C7C700FEFEFEC6C6FEFE85C6C7F81F
:103A000000FEC6C7F8FD0085C7A0F8FA0000C7A0F1
:103A1000A0F800C7C7C7C7C7C7C7C7C7C6C6C7C7F5
:103A2000C7C7C7C7FEFEFEFEFEFEF8FEFEFEFEFE98
:103A3000FBF8FEFEFEFEF8F8F8FEFEFEC7C7C7C69E
:103A4000FEFEC7C60000000000009B009B00C700F0
:103A500000000000C6C7C7C7C7C7C79B009BC7C732
:103A6000C7000000C7C7C6009B00C6C600009B0079
:103A70000085FE009B00FEFEFE000000FEFEFE9B99
:103A8000009BFEFEC7C7C7C7C7C7C79B009BC7C76A
:103A9000C7000000C7C7C6009B00C6C600009B0049
:103AA0000085FE009B00FEFEFE000000FEFEFE9B69
:103AB000009BFEFEC79B009BC7FEC7000000C6FE22
:103AC000C7009B0085FE00009B0000FE85009B0058
:103AD000FEFEFE000000FEFEFE9B009BFEFEFEFEC4
:103AE000FEFEFEFEC6C7C7C7C7C7C79B00C7C7C77E
:103AF000C7000000C7C79B009B00C6C600009B0014
:103B00000085FE009B009BFEFE000000FEFEFEFE08
:103B1000009BFEFEC7C7C7C7C7C7C79B00C7C7C7AD
:103B2000C7000000C7C79B009B00C6C600009B00E3
:103B30000085FE009B009BFEFE000000FEFEFEFED8
:103B4000009BFEFEC79B00C7C7FEC7000000C6FE65
:103B50009B009B0085FE00009B0000FE85009B00F3
:103B60009BFEFE000000FEFEFEFE009BFEFEFEFE33
:103B7000FEFEFEFEC6C7C7C7C7C7C7C700C7C7C7C1
:103B8000C7000000C7C79B009B009BC600009B00AE
:103B900000859B009B009BFEFE000000FEFEFEFEDB
:103BA00000FEFEFEC7C700C7C7C7C7000000C7C7E3
:103BB0009B009B009BC700009B0000C69B009B00D6
:103BC0009B85FE000000FEFEFEFE00FEFEFEFEFEE9
:103BD000FEFEFEFEC7C700C7C7FEC7000000C6FE48
:103BE0009B009B009BFE00009B0000FE9B009B0037
:103BF0009BFEFE000000FEFEFEFE00FEFEFEFEFE40
:103C0000FEFEFEFEC6C7C7C7C7C7C7C7009BC7C75C
:103C1000C7000000C7C7C6009B009BC600009B00F2
:103C200000859B009B00FEFEFE000000FEFEFE9B4A
:103C300000FEFEFEC7C7009BC7C7C7000000C7C77E
:103C4000C7009B009BC700009B0000C69B009B0019
:103C50008585FE000000FEFEFE9B00FEFEFEFEFED1
:103C6000FEFEFEFEC7C7C7C7C7FEC7C7009BC6FE8E
:103C7000C700000085FEC6009B009BFE00009B0065
:103C800000FE9B009B00FEFEFE000000FEFEFE9B71
:103C900000FEFEFEC69B009BC7C7FE000000C7C714
:103CA000FE009B00C7C700009B0000C685009B006C
:103CB0008585FE000000FEFEFE9B009BFEFEFEFED4
:103CC000FEFEFEFEC79B009BC7C7C7000000C7C71C
:103CD000C7009B00C7C700009B0000C685009B0073
:103CE0008585FE000000FEFEFE9B009BFEFEFEFEA4
:103CF000FEFEFEFEC7C7C7C7C7FEC79B009BC6FE2A
:103D0000C700000085FEC6009B0085FE00009B00EA
:103D100000FEFE009B00FEFEFE000000FEFEFE9B7D
:103D2000009BFEFEC69B00C7C7C7C7000000C7C7F1
:103D30009B009B00C7C700009B0000C685009B003E
:103D40009B85FE000000FEFEFEFE009BFEFEFEFECA
:103D5000FEFEFEFEC7C7C7C7C7FEC79B00C7C6FE9D
:103D6000C700000085FE9B009B0085FE00009B00B5
:103D700000FEFE009B009BFEFE000000FEFEFEFE1D
:103D8000009BFEFEC7C7C7C7C7C7C7C700C7C7C70F
:103D9000C7000000C7C79B009B009BC600009B009C
:103DA00000859B009B009BFEFE000000FEFEFEFEC9
:103DB00000FEFEFEC7C7C7C7C7FEC7C700C7C6FE0F
:103DC000C700000085FE9B009B009BFE00009B003F
:103DD00000FE9B009B009BFEFE000000FEFEFEFE20
:103DE00000FEFEFEC7C7C7C7C7C7C7C7009BC7C778
:103DF000C7000000C7C7C6009B009BC600009B0011
:103E000000859B009B00FEFEFE000000FEFEFE9B68
:103E100000FEFEFEFEFEFEFEFE21FEFEFEFE21294F
:103E2000FEFEFEFE2939FEFEFE217939FEFE2169E5
:103E30002969FEFE39297929FE7969792979392993
:103E400039396939FEFEFEFEFEFE61FEFEFEFEFE13
:103E500029FEFEFEFEFE692961FEFE59392961FE3A
:103E60001818697929181859292918182129292178
:103E700018217929FEFEFEFEFEFEFE18FEFEFEFE65
:103E8000592159FEFEFE212921FEFEFE2969392114
:103E9000FEFE61792979FEFE6929692118FE79798A
:103EA00039792118FEFEFEFEFEFEFEFEFEFEFFFE3E
:103EB000FEFEFEFEFFFEFEFEFEFEFFFEFEFEFEFE20
:103EC000FFFEFEFEFEFEFFFEFEFEFEFEFFFEFEFE0F
:103ED000FEFEFFFEFEFEFEFEFEFEFEFEFEFEFEFE01
:103EE000FE0627FEFEFEFEFEFE273FFF06FEFE0646
:103EF0003FFFFEFE27FEFEFEFEFEFEFEFEFEFEFE77
:103F0000FEFEFEFEFEFEFEFEFEFEFEFEFEFEFEFED1
:103F10000627FEFEFEFEFEFE06FE3FFFFE27FE0615
:103F20003FFF27FEFEFEFEFEFEFEFEFEFEFEFEFE46
:103F3000FEFEFEFEFEFEFEFEFEFEFEFEFEFEFEFEA1
:103F400027FEFEFEFEFEFE06FE273FFF27FE06FEC4
:103F50003FFFFE06FEFEFEFEFEFEFEFEFEFEFEFE37
:103F6000FEFEFEFEFEFEFEFEFEF1FEFEFEFEF1F891
:103F7000FEFEFEF107F8FEFE3737F8F8FE373F3F4A
:103F80003FF8373F3F3F3FF1FE3737FEFEFEFE076B
:103F900007FEFEFEFEFEFEFEFEFEF1FEFEFEFEFE45
:103FA00007F1FEFEFEFEF83737FEFEFE3F3F3F37CD
:103FB000FEFE3F3F3F3F37FEFEFE3737FEFEFEFE72
:103FC0000707FEFEFEFEFEFEFE37FEFEFE37373F13
:103FD000FE37373F3F3F373F3F3F3F3F373F3F3F52
:103FE0003F3FFE37373F3F06FEFEFE37373FFEFEC0
:103FF000FEFEFE3737FEFEFEFEFE3F3737FEFEFEBC
:104000003F3F3F3737FE3F3F3F3F3F373F06063F8B
:104010003F37063F3F3737FE3F3737FEFEFE37FE5E
:10402000FEFEFEFEFEFEFEFEFE37FEFEFE37373FC4
:10403000FE37373F3F3F373F3F3F3F3F373F3F3FF1
:10404000063FFE37373F3F06FEFEFE37373FFEFE98
:10405000FEFEFE3737FEFEFEFEFE3F3737FEFEFE5B
:104060003F3F3F3737FE3F3F3F3F3F373F063F3FF2
:104070003F37063F3F3737FE3F3737FEFEFE37FEFE
:10408000FEFEFEFEFEFEFEFEFE37FEFEFE37373F64
:10409000FE37373F3F3F373F3F3F3F3F373F3F06CA
:1040A000063FFE37373F3F06FEFEFE37373FFEFE38
:1040B000FEFEFE3737FEFEFEFEFE3F3737FEFEFEFB
:1040C0003F3F3F3737FE3F3F3F3F3F373F3F3F3F59
:1040D0003F37063F3F3737FE3F3737FEFEFE37FE9E
:1040E000FEFEFEFEFEFEFEFEFEFEFEFEFEFEFEFEF0
:1040F00006FE87FE06FEFE068706FEFEFE06870615
:10410000FEFEFE068706FEFEFEFE87FEFEFEFEFEAD
:1041100087FEFEFEFEFEFEFEFEFEFEFEFEFEFEFE36
:10412000FEFEFEFEFEFEFEFEFEFEFEFEFEFEFEFEAF
:10413000E2FEFEFEFEE2F8E2FEFEFEE2F8E2FEFE37
:10414000FEC0E2C0FEFEFEFEFEFEFEFEFEFEFEFE27
:10415000FEFEFEFEFEFEFEFEE2FEFEFEFEE2F8E2D9
:104160000603FEE2F8E2FEFEFEC0E2C006FEFEFE30
:10417000C0FEFE03FEFEE2FEFEFEFEE2F8E2FEFEF2
:10418000FEE2F8E2FEFE06C0E2C0FEFEFEFEC0FE5B
:10419000FEFEFEFE03FEFEFEFE06FEFEFEFEE2FE4E
:1041A000FEFEFEFEFEFEFEE2FEFEFEFEE2F8E2FE89
:1041B000FEFEE2F8E2FEFEFEC0E2C006FEFEFEC02B
:1041C000FEFEFEFEFE03FEFEFEFEFEFE06FEFEFE02
:1041D000FEFEFEE2FEFEFEFEFEFEFEFEFEFEFEFE1B
:1041E000FEFEFEFEFEFEFEFEFEE2FEFE0306E2F820
:1041F000E2FEFEFEE2F8E2FEFE06C0E2C0FE03FEC4
:10420000FEC0FEFEFEFEFEFEFEC0FEFEFEFE06FE42
:10421000FEFEFE06FEFEFEFEE2FEFEFEFEE2F8E210
:104220000303FEE2F8E2FEFEFEC0E2C0FEFEFEFE7A
:10423000C0FEFEFEFEFEFEFEFEFE06FEFEFEFEFED4
:10424000FE06FEFEFEFEFEFEE2FEFEFE03E2F8E2DB
:10425000FEFEFEE2F8E2FEFEFEC0E2C0FEFEFEFE54
:10426000C0FEFEFEFEFEFEE2F8E2FEFEFEE2F8E228
:10427000FEFEFEC0E2C0FEFEFEFEC0FEFEFEFEFE34
:10428000FEFEFEFEFEFEFEFEFEFEFEFEFEFEFEFE4E
:10429000FEFEFEFEC0C0C0C0C0C03FC0C0C0C0C0A7
:1042A0003FC0C03FC0C03FC0C03FC0C0C03F3F3F95
:1042B0003F3FC03F3FC03F3FC0C03FC03FC0C0C006
:1042C000C0C0C0C0C0C0C0C0C0C03FC0C0C0C0C06F
:1042D0003FC0C0C0C0C03FC0C0C0C0C0C0C0C0C0E0
:1042E000C0C0C0C0C0C0C0C0C0C0C0C0C0C0C0C0CE
:1042F000C0C0C0C0C0C0C0C0C0C0C0070707C0C0E9
:1043000007C0C0C007C007C0C0C007C007C0C0C04A
:1043100007C007C0C0C007C007C0C0C007C0C007F3
:104320000707C0C0C0C0C0C0C0C0C0070707C0C02A
:1043300007C0C0C007C0C0C0C0C007C0C0C007071A
:10434000C0C0C007C0C0C0C007C0C0C0C0C0070751
:10435000070707C0C0C0C0C0C0C0C0070707C0C0B3
:1043600007C0C0C007C0C0C0C0C007C0C0C00707EA
:10437000C0C0C0C0C0C007C007C0C0C007C0C00721
:104380000707C0C0C0C0C0C0C0C007C007C0C0C011
:1043900007C007C0C0C007C007C0C0C007070707E5
:1043A00007C0C0C007C0C0C0C0C007C0C0C0C0C038
:1043B00007C0C0C0C0C0C0C0C0C00707070707C053
:1043C00007C0C0C0C0C007C0C0C0C0C0C00707078A
:1043D000C0C0C0C0C0C007C007C0C0C007C0C007C1
:1043E0000707C0C0C0C0C0C0C0C0C0070707C0C06A
:1043F00007C0C0C007C007C0C0C0C0C007070707CC
:10440000C0C007C0C0C007C007C0C0C007C0C00749
:104410000707C0C0C0C0C0C0C0C0C0C0C0C0C0F8D6
:10442000C0C0C0C0C0F8C0C0C0C0C0F8C0C0C0C01C
:10443000C0F8C0C0C0C0C0F8C0C0C0C0C0F8C0C0D4
:10444000C0C0C0F8C0C0C0C0C0C000000000F8F8C4
:1044500000F8F8F800F800F8F8F800F8000000009C
:10446000F8F800F8F8F8F8F800F8F8F8F8F800F8B4
:10447000F8F8F8F8C0C0C0C0C0C0F8000000F8F8F4
:1044800000F8F8F800F800F8F8F800F800F8F8F884
:1044900000F800F8F8F800F800F8F8F800F8F8006C
:1044A0000000F8F8C0C0C0C0C0C00000000000F8A4
:1044B000F8F800F8F8F8F8F800F8F8F8F8F800F864
:1044C000F8F8F8F800F8F8F8F8F800F8F8F800004C
:1044D000000000F8C0C0C0C0C0C000F8F8F800F884
:1044E0000000F8F800F800F800F800F800F8F8000C
:1044F00000F800F8F8F800F800F8F8F800F800F80C
:10450000F8F800F8C0C0C0C0C0C00000000000F84B
:10451000F8F800F8F8F8F8F800F8F8F8F8F800F803
:10452000F8F8F8F800F8F8F8F8F800F8F8F8F8F8FB
:1045300000F8F8F8C0C0C0C0C0C0F8F8F8F8F8F843
:10454000F8F8F8F8F8F8F8F8F8F8F8F8F8F8F8F8EB
:10455000F8F8F8F8F8F8F8F8F8F8F8F8F8F8F8F8DB
:10456000F8F8F8F8C0C0C0C0C0C0F8000000F8F803
:1045700000F8F8F800F800F8F8F800F8000000007B
:1045800000F800F8F8F800F800F8F8F800F800F87B
:10459000F8F800F8C0C0C0C0C0C0F8F8F8F8F8F8E3
:1045A000F8F80000F8F8F800000000F8000000003B
:1045B0000000000000000000F800000000F8F8F81B
:1045C0000000F8F8C0C0C0C0C0C0C0C0C0C0C0C0FB
:1045D000C0C0C0C0C0C0C0C0C0C0C0C0C0C0C0C0DB
:1045E000C0C0C0C0C0C0C0C0C0C0C0C0C0C0C0C0CB
:1045F000C0C0C0C0C0C0C0C0C0F8C0C0C0C0C0F84B
:10460000C0C0C0C0C0F8C0C0C0C0C0F8C0C0C0C03A
:10461000C0F8C0C0C0C0C0F8C0C0C0C0C0F8C0C0F2
:10462000C0C0C0F8F8F8F8F8F8F8F8F8F8F8F8F8B2
:10463000F8F8F8F8F8F8F8F8F8F8F8F8F8F8F8F8FA
:10464000F8F8F8F8F8F8F8F8F8F8F8F8F8F8F8F8EA
:10465000F8F8F8F8F8F8F8F8F8F8F8F80000F8F8CA
:10466000F800000000F8000000000000000000005A
:104670000000F800000000F8F8F80000F8F8F8F87A
:10468000F8F8F8F8C0C0C0C0C0C0C0C0C0C00707BC
:10469000C0C007070707070707070707073F3F07C8
:1046A0003F3F073F3F073F3FC03F3FC03F3FC0C086
:1046B000C0C0C0C0070707C0C0C0073F0707C0C0D1
:1046C000073F3F07C0C00707070707C0073F3F076F
:1046D00007C0073F3F07C0C0C03F3FC0C0C0C0C009
:1046E000C0C0C0C0C03F3F3FC0C03FC0C0C03FC04F
:1046F000C0C0C0C03FC0C0C03F3FC0C0C03FC0C0BE
:10470000C0C03FC0C0C0C0C03F3F3F3F3FC0C0C0AF
:10471000C0C0C0C0C03FC0C007073F3FC0C007C047
:10472000C03FC0C007C0C03FC0C007C0C03FC0C07E
:104730000707C03FC0C007C03F3F3FC007C0C0C061
:10474000C0C0C0C007C0C0C0C0C0C007C0C0C0C0DB
:10475000C007C0C0C0C0C007C00707C007C0C0C0F6
:10476000C0C0C0C0C0C0C0C0C0C0C0C0C0C0C0C049
:10477000C0C0C0C0C03F3F3FC0C03FC0C0C03FC0BE
:104780003FC0C0C03FC03FC0C0C03FC03FC0C0C0AE
:104790003FC03FC0C0C03FC0C03F3F3FC0C0C0C01F
:1047A000C0C0C0C0C03F3F3FC0C03FC0C0C03FC08E
:1047B000C0C0C0C03FC0C0C03F3FC0C0C0C0C0C07C
:1047C0003FC03FC0C0C03FC0C03F3F3FC0C0C0C0EF
:1047D000C0C0C0C03FC03FC0C0C03FC03FC0C0C0DD
:1047E0003FC03FC0C0C03F3F3F3F3FC0C0C03FC0D1
:1047F000C0C0C0C03FC0C0C0C0C03FC0C0C0C0C0BB
:10480000C0C0C0C03F3F3F3F3FC03FC0C0C0C0C0AE
:104810003FC0C0C0C0C0C03F3F3FC0C0C0C0C0C09C
:104820003FC03FC0C0C03FC0C03F3F3FC0C0C0C08E
:10483000C0C0C0C0C03F3F3FC0C03FC0C0C03FC0FD
:104840003FC0C0C0C0C03F3F3F3FC0C03FC0C0C06E
:104850003FC03FC0C0C03FC0C03F3F3FC0C0C0C05E
:10486000C0C0C0C00707070707F8F8F807F8F8F84E
:10487000F8F807F8F8F8F8F807F8F8F8F8F807F88B
:10488000F8F8F8F807F8F8F8F8F807F8F8F8F8F88A
:10489000F8F8F8F80707070707F8F8F807F8F8F83E
:1048A000F8F807F8F8F8F8F807F8F8F8F8F807F85B
:1048B000F8F8F8F807F8F8F80707070707F8F8F81E
:1048C000F8F8F8F807F8F8F807F80707F80707F80E
:1048D00007F807F807F807F8F8F807F807F8F8F8FE
:1048E00007F807F8F8F807F807F8F8F807F8F8F8FD
:1048F000F8F8F8F80707070707F807F8F8F8F8F8DE
:1049000007F8F8F8F8F8070707F8F8F807F8F8F8DC
:10491000F8F807F8F8F8F8F80707070707F8F8F8BD
:10492000F8F8F8F8F8070707F8F807F8F8F807F8BC
:1049300007F8F8F807F807F8F8F807F807F8F8F8AC
:1049400007F807F8F8F807F8F8070707F8F8F8F88D
:10495000F8F8F8F8F8F80000F8F8F800000000F8A7
:10496000000000000000000000000000F80000004F
:1049700000F8F8F80000F8F8F8F8F8F8F8F8F8F89F
:10498000F8F8F8F8C0C0C0C0C0F8C0C0C0C0C0C00F
:10499000C0C0C0C0C007C0C0C0C0C007C0C0C0C089
:1049A000C007C0C0C0C0C007C0C0C0C0C007C0C032
:1049B000C0C0C0C0F8F8F8F8F8F8C0C0C0C0C0C0A7
:1049C000C0C0C0C0C0C0C0C0C0C0C0C0F8F8F8F807
:1049D000F8F8F8F8F8F8F8F8F8F8F8F8F8F8C0C0C7
:1049E000C0C0C0C0F8F8F8F8F8F8C0C0C0C0C0C077
:1049F000C0C0C0C0C007C0C0C0C0C007F8F8F8F849
:104A0000F807F8F8F8F8F807F8F8F8F8F807C0C069
:104A1000C0C0C0C000FF06015300C00300B0077F44
:104A20000090287F00C10300B1076300911C7F0044
:104A3000C20300B207310092347F00C30000B30705
:104A40002D009305460F075B1190287F00911C7F76
:104A50000092347F0093076711075C1090347F0049
:104A600091287F0092407F009305461107571090D0
:104A7000347F0091287F0092407F0093076210905E
:104A8000327F0091267F00923E7F009307731105CD
:104A9000461090327F0091267F00923E7F00930760
:104AA0005B11902F7F0091237F00923B7F00930743
:104AB000631007651090327F0091267F00923E7F41
:104AC000009305461107751090347F0091287F00F0
:104AD00092407F0093075C1107641090287F00913B
:104AE0001C7F0092347F0093054610077E119028AA
:104AF0007F00911C7F0092347F009307581007605D
:104B00001190347F0091287F0092407F00930546EA
:104B10001007791090347F0091287F0092407F0029
:104B20009307571190327F0091267F00923E7F00BD
:104B30009307661105461090327F0091267F009200
:104B40003E7F0093077410902F7F0091237F009287
:104B50003B7F0093075A11076610902D7F0091212B
:104B60007F0092397F0093054611902E7F0091229D
:104B70007F00923A7F0093077E10902F7F00912351
:104B80007F00923B7F009307591007621190287FA6
:104B900000911C7F0092347F0093054610077F111F
:104BA00090287F00911C7F0092347F0093075B1058
:104BB00007671090347F0091287F0092407F009318
:104BC00005461107781090347F0091287F009240AD
:104BD0007F009307781190327F0091267F00923EEC
:104BE0007F009307571005461090327F0091267F73
:104BF00000923E7F0093077311902F7F0091237FD7
:104C000000923B7F0093077810075B1190327F0082
:104C100091267F00923E7F00930546110765109014
:104C2000347F0091287F0092407F00930775100722
:104C30005C1190287F00911C7F0092347F009305C7
:104C4000461007661190287F00911C7F0092347FE8
:104C50000093077E1007581090347F0091287F0042
:104C600092407F009305461107601090347F0091B9
:104C7000287F0092407F009307791190327F009146
:104C8000267F00923E7F0093075710054610903212
:104C90007F0091267F00923E7F0093077211902F34
:104CA0007F0091237F00923B7F009307741007746D
:104CB00011902D7F0091217F0092397F009305464E
:104CC00010902E7F0091227F00923A7F009307641C
:104CD00010902F7F0091237F00923B7F0093076409
:104CE00011077E10902D7F0091217F0092397F0067
:104CF00093054611076210902D7F0091217F00924D
:104D0000397F0093075F11077F1090397F00912D45
:104D10007F0092457F009305461107671090397F09
:104D200000912D7F0092457F0093075C1090377FA4
:104D300000912B7F0092437F009307781105461066
:104D400090377F00912B7F0092437F009307621181
:104D500090347F0091287F0092407F00930773106A
:104D600007781090377F00912B7F0092437F00934C
:104D700005461107631090397F00912D7F00924501
:104D80007F0093076511077510902D7F0091217F9B
:104D90000092397F0093054610076411902D7F0023
:104DA00091217F0092397F0093076610077E119052
:104DB000397F00912D7F0092457F009305461007B3
:104DC000601090397F00912D7F0092457F009307FE
:104DD000601190377F00912B7F0092437F009307F3
:104DE000601105461090377F00912B7F0092437F22
:104DF000009307571190347F0091287F0092407FE5
:104E0000009307661007721090327F0091267F0092
:104E1000923E7F009305461190337F0091277F00DB
:104E2000923F7F0093075A1090347F0091287F00B3
:104E300092407F009307661107641090287F0091CD
:104E40001C7F0092347F009305461007591190286B
:104E50007F00911C7F0092347F0093076210075FF0
:104E60001190347F0091287F0092407F0093054687
:104E700010075B1090347F0091287F0092407F00E4
:104E80009307671190327F0091267F00923E7F004A
:104E900093075C1005461190327F0091267F0092A7
:104EA0003E7F0093075710902F7F0091237F009241
:104EB0003B7F009307621007731190327F009126A9
:104EC0007F00923E7F0093054611075B1090347F70
:104ED0000091287F0092407F0093076310076511BF
:104EE00090287F00911C7F0092347F00930546102C
:104EF00007751190287F00911C7F0092347F0093EA
:104F0000075C1007641090347F0091287F00924066
:104F10007F0093054611077E1090347F0091287F13
:104F20000092407F009307581190327F0091267FB6
:104F300000923E7F009307601005461090327F007C
:104F400091267F00923E7F0093077911902F7F007A
:104F500091237F00923B7F009307571007661190C3
:104F60002D7F0091217F0092397F0093054610909C
:104F70002E7F0091227F00923A7F00930774109059
:104F80002F7F0091237F00923B7F0093075A1107E8
:104F90006610902F7F0091237F00923B7F00930546
:104FA0004611077E11902F7F0091237F00923B7F57
:104FB000009307590F076211903B7F00912F7F00EC
:104FC00092477F0093054611077F10903B7F009129
:104FD0002F7F0092477F0093075B1190397F0091EC
:104FE0002D7F0092457F009307671005461090398A
:104FF0007F00912D7F0092457F00930778119036B6
:105000007F00912A7F0092427F0093077810075714
:105010001190397F00912D7F0092457F00930546C6
:1050200010077310903B7F00912F7F0092477F0005
:1050300093077811075B10902D7F0091217F0092DC
:10504000397F0093054611076510902D7F0091214F
:105050007F0092397F0093077510075C1190397FAC
:1050600000912D7F0092457F009305461007661141
:1050700090397F00912D7F0092457F0093077E102D
:1050800090377F00912B7F0092437F009307581148
:1050900005461090377F00912B7F0092437F00934D
:1050A00007601190347F0091287F0092407F009329
:1050B00007791007571090377F00912B7F0092439C
:1050C0007F009305461107721090397F00912D7F64
:1050D0000092457F009307741107741090287F0099
:1050E000911C7F0092347F00930546100764119055
:1050F000287F00911C7F0092347F00930764100783
:105100007E1190347F0091287F0092407F009305AC
:10511000461007621090347F0091287F0092407FF4
:105120000093075F1190327F0091267F00923E7FAF
:105130000093077F1005461190327F0091267F0073
:10514000923E7F0093076710902F7F0091237F008E
:10515000923B7F0093075C1007781190327F00919B
:10516000267F00923E7F009305461107621090341F
:105170007F0091287F0092407F009307731107788A
:105180001090287F00911C7F0092347F0093054689
:105190001090287F00911C7F0092347F009307635A
:1051A0001107651090287F00911C7F0092347F00CA
:1051B00093077511902C7F0091207F0092387F001B
:1051C00093054610902C7F0091207F0092387F003D
:1051D00093076410076611902C7F0091207F009246
:1051E000387F0093077E10902D7F0091217F0092E1
:1051F000397F0093054611902D7F0091217F009209
:10520000397F0093076010076010902D7F00912177
:105210007F0092397F0093076011902E7F009122CA
:105220007F00923A7F0093054610902E7F009122D6
:105230007F00923A7F0093075711076610902F7FE7
:105240000091237F00923B7F0093077210FF0601BD
:105250004500FF2F000002060000FB00FF0000F4E5
:1052600005030C05040C05030C05040C05050000E2
:10527000FF00FF0002090000F10400F900FF000137
:105280000A0000E20201050101030101010205001B
:1052900000FF0000E702030C04050000FF0000F11E
:1052A00000085A0204030204040204050204060270
:1052B000050000FF0001010007900000E208050062
:1052C00000FF0002080107C80106000100E700FF17
:1052D0000001000007A00000EC0100FE0001010039
:1052E000FF0001030000E2030106040109030500B9
:1052F00000FF0002010107C80106000100EC00FFE9
:105300000002040000F10400F900FF0002010000A7
:10531000F100FF0000ED00010602010100FF0000A6
:10532000EC0001020107000207FF00010300FF007B
:1053300002080007640100140500F700FF000209DD
:105340000000F100FF0002040000F800085003080C
:105350004E03085402084C02085802084A01085C2F
:105360000000FC03086003085A03086003085A039E
:10537000086003085A01050000FF0002040000FB5A
:1053800000083E01030201030201030201030201BE
:10539000030201040A0103020103020103020103E3
:1053A00002010302010402010302010302010302DC
:1053B00001030201030201040A01030201030201C5
:1053C00003020103020103020104050103020103B8
:1053D00002010302010302010302010405010302A9
:1053E000010302010302010302010302010405019A
:1053F000030201030201030201030201030201058A
:105400000000FF00020300085602040A020408021A
:105410000406020404020402000842020305020416
:10542000020203050203050204020203050000F85C
:10543000040305040405040305040405040305042A
:10544000040504030501050000FF0002040000FB41
:1054500000083401030201030401030601040A01E8
:10546000030201030401030601040A01030201030C
:1054700004010306010405010302010304010306FC
:1054800002030202030402030603040503030203EA
:1054900003040303060404050403020403040403D1
:1054A0000601050000FF0007000402040007FF00DA
:1054B0000990000A3C0000FB0108500303050304A7
:1054C000050303050304050303050304050303059E
:1054D000030405030305030405030305030405038F
:1054E000030503050000FF0007000402040007FF96
:1054F000000990000A3C0000FB0108530303050368
:10550000040503030503040503030503040503035E
:10551000050304050303050304050303050304054C
:1055200003030503050000FF000700040204000751
:10553000FF000990000A3C0000FB01085603030528
:10554000030405030305030405030305030405031E
:10555000030503040503030503040503030503040E
:105560000503030503050000FF0007000402040013
:1055700007FF000990000A3C0000FB0108590303E3
:1055800005030405030305030405030305030405DC
:1055900003030503040503030503040503030503CF
:1055A000040503030503050000FF000202010600D5
:1055B0000100E000FF0002010106000100E000FF21
:1055C0000002080106000100E000FF0002050106DC
:1055D000000100E000FF0002090106000100E000F8
:1055E000FF0000005552000000000000005D520066
:1055F0000000000000007152000000000000007375
:1056000052000000000100007E5200000000000077
:10561000009252000000000000009D5200000000B7
:10562000010000B45200000000000000C25200005F
:105630000000010000D05200000000010000E15213
:1056400000000000000000F2520000000000000016
:105650000053000000000000000B53000000000198
:1056600000001353000000000100001E5300000062
:10567000000000002F53000000000000003D530018
:105680000000000000004553000000000000007A08
:105690005300000000000000035400000000000060
:1056A000004A5400000000000000A6540000000062
:1056B000000000E754000000000000002855000032
:1056C0000000000000695500000000000000AA551D
:1056D00000000000000000B55500000000000000C0
:1056E000C05500000000000000CB55000000000085
:1056F0000000D6550000000005060708090A0B0C3B
:105700000D0E0F101112131409150B16170E181089
:105710002223242526272425010101000000FF0063
:10572000FF00000100000000FF0000010001000078
:105730000100FFFF00000100FFFEFDFCFBFAF9F78E
:10574000F7F5F5F4F3F2F1F1EFEFEEEDEDEDECEB53
:10575000EBEBEBEAEAEAEAEAEAEAEAEAEAEBEBEBA3
:10576000ECECEDEDEEEFEFF0F1F2F3F3F5F5F7F72A
:10577000F9F9FBFBFDFDFF00323436393B3E404278
:105780004547494B4D4F51535557585A5B5C5E5FE7
:1057900060616162636363636463636363626161E5
:1057A000605F5E5C5B5A58575553514F4D4B4947AC
:1057B0004542403E3B393634322F2D2A28252321BD
:1057C0001E1C1A18161412100E0C0B0908070504DB
:1057D00003020201000000000000000000010202BC
:1057E0000304050708090B0C0E10121416181A1CD6
:1057F0001E212325282A2D2F646363636362616160
:10580000605F5E5C5B5A58575553514F4D4B49474B
:105810004542403E3B393634322F2D2A282523215C
:105820001E1C1A18161412100E0C0B09080705047A
:10583000030202010000000000000000000102025B
:105840000304050708090B0C0E10121416181A1C75
:105850001E212325282A2D2F313436393B3E404244
:105860004547494B4D4F51535557585A5B5C5E5F06
:105870006061616263636363060201000203040501
:1058800006070800080001000602000601000600E5
:1058900008080E06060E06060607020304050108A0
:1058A000080011241FBECFEFD0E1DEBFCDBF14BE74
:1058B00088E10FB6F89480936000109260000FBEEC
:1058C00011E0A0E0B1E0EAEEFEEA02C005900D9220
:1058D000A43AB107D9F71FE0A4EAB1E001C01D92D4
:1058E000A131B107E1F7F894E1E2FCE080E090E05B
:1058F00020E802C02193019632E08C309307D4F364
:1059000081E29CE090932E0E80932D0E10922F0E2C
:10591000E2E3FEE080E090E003C0108201963A9658
:1059200084309105D4F381E08093520E8093530E1E
:105930008093510E1092810015BCE0E0F1E080E010
:1059400090E02EEF02C02193019680399105DCF39F
:1059500090936C0E80936B0E80E00E949844E0E080
:10596000F7E080E090E050ED20EC31E041E00EC047
:1059700010821182009719F45093020701C012821D
:10598000348323831782408701963F968F30910599
:105990007CF390936C0E80936B0E91E09093F90BD7
:1059A0008FEF87B984B980E88AB98CE081B983EF39
:1059B00082B91092FA0B86E08093FB0B109285005F
:1059C0001092840083E0809389008DE880938800A2
:1059D00089E08093810082E080936F0082E484BD3F
:1059E00017BC95BD83E88093B0001092B3009093EC
:1059F000B10081E185B978940E948C450E94895557
:105A00000C9473570C9400002C44364444444F4388
:105A1000EBEDC8950000EA95E1F700C000C04091A9
:105A20000507509106074ABD5BBDC0910B07D09199
:105A30000C0740900D0750900E0790900707F090CC
:105A40000207E0900A0770910107672F67708824AA
:105A500000EDA02EA4EEB7E075D00027E101D30140
:105A600008B9F1E0E091F40B1193119311931193A4
:105A700011931193E091F50B1193119311931193DD
:105A800011931193E091F60B1193119311931193CC
:105A900011931193E091F70B1193119311931193BB
:105AA00011931193E091F80B1193119311931193AA
:105AB0001193119363957395FA94A9F483940FE06D
:105AC000809EF001E050F94F058016800ABC1BBC97
:105AD000C385D485458456849780F280E2847181A1
:105AE000672F677008C00000000000000000000081
:105AF00009E00A95F1F7791509F4E20109F477272D
:105B000009F46627AA9441F0683019F000C000C07B
:105B1000A3CF6627A096A0CFC895C8950E941D4424
:105B20004091FB0B405D4093FB0B11E00091FD0B9E
:105B300001270093FD0BE1E0E093FC0BE2E0E09332
:105B4000360008952898E0912D0EF0912E0E0191C7
:105B50002EE0ED32F20721E23CE00093B30008F0C2
:105B6000F901E0932D0EF0932E0E1E01C090E20776
:105B7000D090E30780E323E036E0D1E040EA56E04E
:105B800098E00D91099F112D0F71FA01029FE00D10
:105B9000F11D0281C081F601089FE00DF11D139FE8
:105BA000E00DF11DC093F40B059009920590099248
:105BB0000590099205900992059009920590099225
:105BC0000D91099F112D0F71FA01029FE00DF11D3A
:105BD0000281C081F601089FE00DF11D139FE00DC9
:105BE000F11DC093F50B059009920590099205905F
:105BF0000992059009920D91289A059009920590B5
:105C00000992099F112D0F71FA01029FE00DF11DFC
:105C10000281C081F601089FE00DF11D139FE00D88
:105C2000F11DC093F60B059009920590099205901D
:105C300009920590099205900992059009920D919B
:105C4000099F112D0F71FA01029FE00DF11D0281D4
:105C5000C081F601089FE00DF11D139FE00DF11DBD
:105C6000C093F70B0590099205900992059009924F
:105C70000590099205900992059009920D91099F4E
:105C8000112D0F71FA01029FE00DF11D0281C081FB
:105C9000F601089FE00DF11D139FE00DF11DC0936B
:105CA000F80B0590099205900992059009920590CC
:105CB00009920590099205900992E1013D01DE01EA
:105CC0001EEF4AB55BB5639FC0013A2F307ECE2DE3
:105CD000CC0FDD27C057DE4FE991F881C6E0D1E057
:105CE000CC9020E3C29EA395AF71A32B040E151E8A
:105CF000080E191E0994F001C895C895C895C89555
:105D00000591D990D1120D2D08B9CC900591D9905B
:105D1000D1120D2D08B9C29E0591D990D1120D2D29
:105D200008B9040E151E0591D990D1120D2D08B990
:105D3000080E191E0591D990D1120D2D08B9A39501
:105D4000AF710591D990D1120D2D08B9A32BF00197
:105D50000591D990D1120D2D08B9CC900591D9900B
:105D6000D1120D2D08B9C29E0591D990D1120D2DD9
:105D700008B9040E151E0591D990D1120D2D08B940
:105D8000080E191E0591D990D1120D2D08B9A395B1
:105D9000AF710591D990D1120D2D08B9A32BF00147
:105DA0000591D990D1120D2D08B9CC900591D990BB
:105DB000D1120D2D08B9C29E0591D990D1120D2D89
:105DC00008B9040E151E0591D990D1120D2D08B9F0
:105DD000080E191E0591D990D1120D2D08B9A39561
:105DE000AF710591D990D1120D2D08B9A32BF001F7
:105DF0000591D990D1120D2D08B9CC900591D9906B
:105E0000D1120D2D08B9C29E0591D990D1120D2D38
:105E100008B9040E151E0591D990D1120D2D08B99F
:105E2000080E191E0591D990D1120D2D08B9A39510
:105E3000AF710591D990D1120D2D08B9A32BF001A6
:105E40000591D990D1120D2D08B9CC900591D9901A
:105E5000D1120D2D08B9C29E0591D990D1120D2DE8
:105E600008B9040E151E0591D990D1120D2D08B94F
:105E7000080E191E0591D990D1120D2D08B9A395C0
:105E8000AF710591D990D1120D2D08B9A32BF00156
:105E90000591D990D1120D2D08B9CC900591D990CA
:105EA000D1120D2D08B9C29E0591D990D1120D2D98
:105EB00008B9040E151E0591D990D1120D2D08B9FF
:105EC000080E191E0591D990D1120D2D08B9A39570
:105ED000AF710591D990D1120D2D08B9A32BF00106
:105EE0000591D990D1120D2D08B9CC900591D9907A
:105EF000D1120D2D08B9C29E0591D990D1120D2D48
:105F000008B9040E151E0591D990D1120D2D08B9AE
:105F1000080E191E0591D990D1120D2D08B9A3951F
:105F2000AF710591D990D1120D2D08B9A32BF001B5
:105F30000591D990D1120D2D08B9CC900591D99029
:105F4000D1120D2D08B9C29E0591D990D1120D2DF7
:105F500008B9040E151E0591D990D1120D2D08B95E
:105F6000080E191E0591D990D1120D2D08B9A395CF
:105F7000AF710591D990D1120D2D08B9A32BF00165
:105F80000591D990D1120D2D08B9CC900591D990D9
:105F9000D1120D2D08B9C29E0591D990D1120D2DA7
:105FA00008B9040E151E0591D990D1120D2D08B90E
:105FB000080E191E0591D990D1120D2D08B9A3957F
:105FC000AF710591D990D1120D2D08B9A32BF00115
:105FD0000591D990D1120D2D08B9CC900591D99089
:105FE000D1120D2D08B9C29E0591D990D1120D2D57
:105FF00008B9040E151E0591D990D1120D2D08B9BE
:10600000080E191E0591D990D1120D2D08B9A3952E
:10601000AF710591D990D1120D2D08B9A32BF001C4
:106020000591D990D1120D2D08B9CC900591D99038
:10603000D1120D2D08B9C29E0591D990D1120D2D06
:1060400008B9040E151E0591D990D1120D2D08B96D
:10605000080E191E0591D990D1120D2D08B9A395DE
:10606000AF710591D990D1120D2D08B9A32BF00174
:106070000591D990D1120D2D08B9CC900591D990E8
:10608000D1120D2D08B9C29E0591D990D1120D2DB6
:1060900008B9040E151E0591D990D1120D2D08B91D
:1060A000080E191E0591D990D1120D2D08B9A3958E
:1060B000AF710591D990D1120D2D08B9A32BF00124
:1060C0000591D990D1120D2D08B9CC900591D99098
:1060D000D1120D2D08B9C29E0591D990D1120D2D66
:1060E00008B9040E151E0591D990D1120D2D08B9CD
:1060F000080E191E0591D990D1120D2D08B9A3953E
:10610000AF710591D990D1120D2D08B9A32BF001D3
:106110000591D990D1120D2D08B9CC900591D99047
:10612000D1120D2D08B9C29E0591D990D1120D2D15
:1061300008B9040E151E0591D990D1120D2D08B97C
:10614000080E191E0591D990D1120D2D08B9A395ED
:10615000AF710591D990D1120D2D08B9A32BF00183
:106160000591D990D1120D2D08B9CC900591D990F7
:10617000D1120D2D08B9C29E0591D990D1120D2DC5
:1061800008B9040E151E0591D990D1120D2D08B92C
:10619000080E191E0591D990D1120D2D08B9A3959D
:1061A000AF710591D990D1120D2D08B9A32BF00133
:1061B0000591D990D1120D2D08B9CC900591D990A7
:1061C000D1120D2D08B9C29E0591D990D1120D2D75
:1061D00008B9040E151E0591D990D1120D2D08B9DC
:1061E000080E191E0591D990D1120D2D08B9A3954D
:1061F000AF710591D990D1120D2D08B9A32BF001E3
:106200000591D990D1120D2D08B9CC900591D99056
:10621000D1120D2D08B9C29E0591D990D1120D2D24
:1062200008B9040E151E0591D990D1120D2D08B98B
:10623000080E191E0591D990D1120D2D08B9A395FC
:10624000AF710591D990D1120D2D08B9A32BF00192
:106250000591D990D1120D2D08B9CC900591D99006
:10626000D1120D2D08B9C29E0591D990D1120D2DD4
:1062700008B9040E151E0591D990D1120D2D08B93B
:10628000080E191E0591D990D1120D2D08B9A395AC
:10629000AF710591D990D1120D2D08B9A32BF00142
:1062A0000591D990D1120D2D08B9CC900591D990B6
:1062B000D1120D2D08B9C29E0591D990D1120D2D84
:1062C00008B9040E151E0591D990D1120D2D08B9EB
:1062D000080E191E0591D990D1120D2D08B9A3955C
:1062E000AF710591D990D1120D2D08B9A32BF001F2
:1062F0000591D990D1120D2D08B9CC900591D99066
:10630000D1120D2D08B9C29E0591D990D1120D2D33
:1063100008B9040E151E0591D990D1120D2D08B99A
:10632000080E191E0591D990D1120D2D08B9A3950B
:10633000AF710591D990D1120D2D08B9A32BF001A1
:106340000591D990D1120D2D08B9CC900591D99015
:10635000D1120D2D08B9C29E0591D990D1120D2DE3
:1063600008B9040E151E0591D990D1120D2D08B94A
:10637000080E191E0591D990D1120D2D08B9A395BB
:10638000AF710591D990D1120D2D08B9A32BF00151
:106390000591D990D1120D2D08B9CC900591D990C5
:1063A000D1120D2D08B9C29E0591D990D1120D2D93
:1063B00008B9040E151E0591D990D1120D2D08B9FA
:1063C000080E191E0591D990D1120D2D08B9A3956B
:1063D000AF710591D990D1120D2D08B9A32BF00101
:1063E0000895F0013196CC9000C000C000C000C0FC
:1063F0000591D990D1120D2D08B9C29E0591D99061
:10640000D1120D2D08B9040E151E0591D990D11287
:106410000D2D08B9080E191E0591D990D1120D2D18
:1064200008B9A395AF710591D990D1120D2D08B976
:10643000A32BF0010591D990D1120D2D08B9CC9064
:106440000591D990D1120D2D08B9C29E0591D99010
:10645000D1120D2D08B9040E151E0591D990D11237
:106460000D2D08B9080E191E0591D990D1120D2DC8
:1064700008B9A395AF710591D990D1120D2D08B926
:10648000A32BF0010591D990D1120D2D08B9CC9014
:106490000591D990D1120D2D08B9C29E0591D990C0
:1064A000D1120D2D08B9040E151E0591D990D112E7
:1064B0000D2D08B9080E191E0591D990D1120D2D78
:1064C00008B9A395AF710591D990D1120D2D08B9D6
:1064D000A32BF0010591D990D1120D2D08B9CC90C4
:1064E0000591D990D1120D2D08B9C29E0591D99070
:1064F000D1120D2D08B9040E151E0591D990D11297
:106500000D2D08B9080E191E0591D990D1120D2D27
:1065100008B9A395AF710591D990D1120D2D08B985
:10652000A32BF0010591D990D1120D2D08B9CC9073
:106530000591D990D1120D2D08B9C29E0591D9901F
:10654000D1120D2D08B9040E151E0591D990D11246
:106550000D2D08B9080E191E0591D990D1120D2DD7
:1065600008B9A395AF710591D990D1120D2D08B935
:10657000A32BF0010591D990D1120D2D08B9CC9023
:106580000591D990D1120D2D08B9C29E0591D990CF
:10659000D1120D2D08B9040E151E0591D990D112F6
:1065A0000D2D08B9080E191E0591D990D1120D2D87
:1065B00008B9A395AF710591D990D1120D2D08B9E5
:1065C000A32BF0010591D990D1120D2D08B9CC90D3
:1065D0000591D990D1120D2D08B9C29E0591D9907F
:1065E000D1120D2D08B9040E151E0591D990D112A6
:1065F0000D2D08B9080E191E0591D990D1120D2D37
:1066000008B9A395AF710591D990D1120D2D08B994
:10661000A32BF0010591D990D1120D2D08B9CC9082
:106620000591D990D1120D2D08B9C29E0591D9902E
:10663000D1120D2D08B9040E151E0591D990D11255
:106640000D2D08B9080E191E0591D990D1120D2DE6
:1066500008B9A395AF710591D990D1120D2D08B944
:10666000A32BF0010591D990D1120D2D08B9CC9032
:106670000591D990D1120D2D08B9C29E0591D990DE
:10668000D1120D2D08B9040E151E0591D990D11205
:106690000D2D08B9080E191E0591D990D1120D2D96
:1066A00008B9A395AF710591D990D1120D2D08B9F4
:1066B000A32BF0010591D990D1120D2D08B9CC90E2
:1066C0000591D990D1120D2D08B9C29E0591D9908E
:1066D000D1120D2D08B9040E151E0591D990D112B5
:1066E0000D2D08B9080E191E0591D990D1120D2D46
:1066F00008B9A395AF710591D990D1120D2D08B9A4
:10670000A32BF0010591D990D1120D2D08B9CC9091
:106710000591D990D1120D2D08B9C29E0591D9903D
:10672000D1120D2D08B9040E151E0591D990D11264
:106730000D2D08B9080E191E0591D990D1120D2DF5
:1067400008B9A395AF710591D990D1120D2D08B953
:10675000A32BF0010591D990D1120D2D08B9CC9041
:106760000591D990D1120D2D08B9C29E0591D990ED
:10677000D1120D2D08B9040E151E0591D990D11214
:106780000D2D08B9080E191E0591D990D1120D2DA5
:1067900008B9A395AF710591D990D1120D2D08B903
:1067A000A32BF0010591D990D1120D2D08B9CC90F1
:1067B0000591D990D1120D2D08B9C29E0591D9909D
:1067C000D1120D2D08B9040E151E0591D990D112C4
:1067D0000D2D08B9080E191E0591D990D1120D2D55
:1067E00008B9A395AF710591D990D1120D2D08B9B3
:1067F000A32BF0010591D990D1120D2D08B9CC90A1
:106800000591D990D1120D2D08B9C29E0591D9904C
:10681000D1120D2D08B9040E151E0591D990D11273
:106820000D2D08B9080E191E0591D990D1120D2D04
:1068300008B9A395AF710591D990D1120D2D08B962
:10684000A32BF0010591D990D1120D2D08B9CC9050
:106850000591D990D1120D2D08B9C29E0591D990FC
:10686000D1120D2D08B9040E151E0591D990D11223
:106870000D2D08B9080E191E0591D990D1120D2DB4
:1068800008B9A395AF710591D990D1120D2D08B912
:10689000A32BF0010591D990D1120D2D08B9CC9000
:1068A0000591D990D1120D2D08B9C29E0591D990AC
:1068B000D1120D2D08B9040E151E0591D990D112D3
:1068C0000D2D08B9080E191E0591D990D1120D2D64
:1068D00008B9A395AF710591D990D1120D2D08B9C2
:1068E000A32BF0010591D990D1120D2D08B9CC90B0
:1068F0000591D990D1120D2D08B9C29E0591D9905C
:10690000D1120D2D08B9040E151E0591D990D11282
:106910000D2D08B9080E191E0591D990D1120D2D13
:1069200008B9A395AF710591D990D1120D2D08B971
:10693000A32BF0010591D990D1120D2D08B9CC905F
:106940000591D990D1120D2D08B9C29E0591D9900B
:10695000D1120D2D08B9040E151E0591D990D11232
:106960000D2D08B9080E191E0591D990D1120D2DC3
:1069700008B9A395AF710591D990D1120D2D08B921
:10698000A32BF0010591D990D1120D2D08B9CC900F
:106990000591D990D1120D2D08B9C29E0591D990BB
:1069A000D1120D2D08B9040E151E0591D990D112E2
:1069B0000D2D08B9080E191E0591D990D1120D2D73
:1069C00008B9A395AF710591D990D1120D2D08B9D1
:1069D000A32BF0010591D990D1120D2D08B9CC90BF
:1069E0000591D990D1120D2D08B9C29E0591D9906B
:1069F000D1120D2D08B9040E151E0591D990D11292
:106A00000D2D08B9080E191E0591D990D1120D2D22
:106A100008B9A395AF710591D990D1120D2D08B980
:106A2000A32BF0010591D990D1120D2D08B9CC906E
:106A30000591D990D1120D2D08B9C29E0591D9901A
:106A4000D1120D2D08B9040E151E0591D990D11241
:106A50000D2D08B9080E191E0591D990D1120D2DD2
:106A600008B9A395AF710591D990D1120D2D08B930
:106A7000A32BF0010591D990D1120D2D08B9CC901E
:106A80000591D990D1120D2D08B9C29E0591D990CA
:106A9000D1120D2D08B9040E151E0591D990D112F1
:106AA0000D2D08B9080E191E0591D990D1120D2D82
:106AB00008B9A395AF710591D990D1120D2D08B9E0
:106AC000A32BF0010591D990D1120D2D08B9CC90CE
:106AD0000895F0013296CC90C29E00C000C000C064
:106AE0000591D990D1120D2D08B9040E151E0591EE
:106AF000D990D1120D2D08B9080E191E0591D99003
:106B0000D1120D2D08B9A395AF710591D990D1126D
:106B10000D2D08B9A32BF0010591D990D1120D2D9F
:106B200008B9CC900591D990D1120D2D08B9C29E0B
:106B30000591D990D1120D2D08B9040E151E05919D
:106B4000D990D1120D2D08B9080E191E0591D990B2
:106B5000D1120D2D08B9A395AF710591D990D1121D
:106B60000D2D08B9A32BF0010591D990D1120D2D4F
:106B700008B9CC900591D990D1120D2D08B9C29EBB
:106B80000591D990D1120D2D08B9040E151E05914D
:106B9000D990D1120D2D08B9080E191E0591D99062
:106BA000D1120D2D08B9A395AF710591D990D112CD
:106BB0000D2D08B9A32BF0010591D990D1120D2DFF
:106BC00008B9CC900591D990D1120D2D08B9C29E6B
:106BD0000591D990D1120D2D08B9040E151E0591FD
:106BE000D990D1120D2D08B9080E191E0591D99012
:106BF000D1120D2D08B9A395AF710591D990D1127D
:106C00000D2D08B9A32BF0010591D990D1120D2DAE
:106C100008B9CC900591D990D1120D2D08B9C29E1A
:106C20000591D990D1120D2D08B9040E151E0591AC
:106C3000D990D1120D2D08B9080E191E0591D990C1
:106C4000D1120D2D08B9A395AF710591D990D1122C
:106C50000D2D08B9A32BF0010591D990D1120D2D5E
:106C600008B9CC900591D990D1120D2D08B9C29ECA
:106C70000591D990D1120D2D08B9040E151E05915C
:106C8000D990D1120D2D08B9080E191E0591D99071
:106C9000D1120D2D08B9A395AF710591D990D112DC
:106CA0000D2D08B9A32BF0010591D990D1120D2D0E
:106CB00008B9CC900591D990D1120D2D08B9C29E7A
:106CC0000591D990D1120D2D08B9040E151E05910C
:106CD000D990D1120D2D08B9080E191E0591D99021
:106CE000D1120D2D08B9A395AF710591D990D1128C
:106CF0000D2D08B9A32BF0010591D990D1120D2DBE
:106D000008B9CC900591D990D1120D2D08B9C29E29
:106D10000591D990D1120D2D08B9040E151E0591BB
:106D2000D990D1120D2D08B9080E191E0591D990D0
:106D3000D1120D2D08B9A395AF710591D990D1123B
:106D40000D2D08B9A32BF0010591D990D1120D2D6D
:106D500008B9CC900591D990D1120D2D08B9C29ED9
:106D60000591D990D1120D2D08B9040E151E05916B
:106D7000D990D1120D2D08B9080E191E0591D99080
:106D8000D1120D2D08B9A395AF710591D990D112EB
:106D90000D2D08B9A32BF0010591D990D1120D2D1D
:106DA00008B9CC900591D990D1120D2D08B9C29E89
:106DB0000591D990D1120D2D08B9040E151E05911B
:106DC000D990D1120D2D08B9080E191E0591D99030
:106DD000D1120D2D08B9A395AF710591D990D1129B
:106DE0000D2D08B9A32BF0010591D990D1120D2DCD
:106DF00008B9CC900591D990D1120D2D08B9C29E39
:106E00000591D990D1120D2D08B9040E151E0591CA
:106E1000D990D1120D2D08B9080E191E0591D990DF
:106E2000D1120D2D08B9A395AF710591D990D1124A
:106E30000D2D08B9A32BF0010591D990D1120D2D7C
:106E400008B9CC900591D990D1120D2D08B9C29EE8
:106E50000591D990D1120D2D08B9040E151E05917A
:106E6000D990D1120D2D08B9080E191E0591D9908F
:106E7000D1120D2D08B9A395AF710591D990D112FA
:106E80000D2D08B9A32BF0010591D990D1120D2D2C
:106E900008B9CC900591D990D1120D2D08B9C29E98
:106EA0000591D990D1120D2D08B9040E151E05912A
:106EB000D990D1120D2D08B9080E191E0591D9903F
:106EC000D1120D2D08B9A395AF710591D990D112AA
:106ED0000D2D08B9A32BF0010591D990D1120D2DDC
:106EE00008B9CC900591D990D1120D2D08B9C29E48
:106EF0000591D990D1120D2D08B9040E151E0591DA
:106F0000D990D1120D2D08B9080E191E0591D990EE
:106F1000D1120D2D08B9A395AF710591D990D11259
:106F20000D2D08B9A32BF0010591D990D1120D2D8B
:106F300008B9CC900591D990D1120D2D08B9C29EF7
:106F40000591D990D1120D2D08B9040E151E059189
:106F5000D990D1120D2D08B9080E191E0591D9909E
:106F6000D1120D2D08B9A395AF710591D990D11209
:106F70000D2D08B9A32BF0010591D990D1120D2D3B
:106F800008B9CC900591D990D1120D2D08B9C29EA7
:106F90000591D990D1120D2D08B9040E151E059139
:106FA000D990D1120D2D08B9080E191E0591D9904E
:106FB000D1120D2D08B9A395AF710591D990D112B9
:106FC0000D2D08B9A32BF0010591D990D1120D2DEB
:106FD00008B9CC900591D990D1120D2D08B9C29E57
:106FE0000591D990D1120D2D08B9040E151E0591E9
:106FF000D990D1120D2D08B9080E191E0591D990FE
:10700000D1120D2D08B9A395AF710591D990D11268
:107010000D2D08B9A32BF0010591D990D1120D2D9A
:1070200008B9CC900591D990D1120D2D08B9C29E06
:107030000591D990D1120D2D08B9040E151E059198
:10704000D990D1120D2D08B9080E191E0591D990AD
:10705000D1120D2D08B9A395AF710591D990D11218
:107060000D2D08B9A32BF0010591D990D1120D2D4A
:1070700008B9CC900591D990D1120D2D08B9C29EB6
:107080000591D990D1120D2D08B9040E151E059148
:10709000D990D1120D2D08B9080E191E0591D9905D
:1070A000D1120D2D08B9A395AF710591D990D112C8
:1070B0000D2D08B9A32BF0010591D990D1120D2DFA
:1070C00008B9CC900591D990D1120D2D08B9C29E66
:1070D0000591D990D1120D2D08B9040E151E0591F8
:1070E000D990D1120D2D08B9080E191E0591D9900D
:1070F000D1120D2D08B9A395AF710591D990D11278
:107100000D2D08B9A32BF0010591D990D1120D2DA9
:1071100008B9CC900591D990D1120D2D08B9C29E15
:107120000591D990D1120D2D08B9040E151E0591A7
:10713000D990D1120D2D08B9080E191E0591D990BC
:10714000D1120D2D08B9A395AF710591D990D11227
:107150000D2D08B9A32BF0010591D990D1120D2D59
:1071600008B9CC900591D990D1120D2D08B9C29EC5
:107170000591D990D1120D2D08B9040E151E059157
:10718000D990D1120D2D08B9080E191E0591D9906C
:10719000D1120D2D08B9A395AF710591D990D112D7
:1071A0000D2D08B9A32BF0010591D990D1120D2D09
:1071B00008B9CC900591D990D1120D2D08B9C29E75
:1071C0000895F0013396CC90C29E040E151E00C0A7
:1071D00000C00591D990D1120D2D08B9080E191EC5
:1071E0000591D990D1120D2D08B9A395AF710591D4
:1071F000D990D1120D2D08B9A32BF0010591D9908A
:10720000D1120D2D08B9CC900591D990D1120D2D28
:1072100008B9C29E0591D990D1120D2D08B9040E5E
:10722000151E0591D990D1120D2D08B9080E191E01
:107230000591D990D1120D2D08B9A395AF71059183
:10724000D990D1120D2D08B9A32BF0010591D99039
:10725000D1120D2D08B9CC900591D990D1120D2DD8
:1072600008B9C29E0591D990D1120D2D08B9040E0E
:10727000151E0591D990D1120D2D08B9080E191EB1
:107280000591D990D1120D2D08B9A395AF71059133
:10729000D990D1120D2D08B9A32BF0010591D990E9
:1072A000D1120D2D08B9CC900591D990D1120D2D88
:1072B00008B9C29E0591D990D1120D2D08B9040EBE
:1072C000151E0591D990D1120D2D08B9080E191E61
:1072D0000591D990D1120D2D08B9A395AF710591E3
:1072E000D990D1120D2D08B9A32BF0010591D99099
:1072F000D1120D2D08B9CC900591D990D1120D2D38
:1073000008B9C29E0591D990D1120D2D08B9040E6D
:10731000151E0591D990D1120D2D08B9080E191E10
:107320000591D990D1120D2D08B9A395AF71059192
:10733000D990D1120D2D08B9A32BF0010591D99048
:10734000D1120D2D08B9CC900591D990D1120D2DE7
:1073500008B9C29E0591D990D1120D2D08B9040E1D
:10736000151E0591D990D1120D2D08B9080E191EC0
:107370000591D990D1120D2D08B9A395AF71059142
:10738000D990D1120D2D08B9A32BF0010591D990F8
:10739000D1120D2D08B9CC900591D990D1120D2D97
:1073A00008B9C29E0591D990D1120D2D08B9040ECD
:1073B000151E0591D990D1120D2D08B9080E191E70
:1073C0000591D990D1120D2D08B9A395AF710591F2
:1073D000D990D1120D2D08B9A32BF0010591D990A8
:1073E000D1120D2D08B9CC900591D990D1120D2D47
:1073F00008B9C29E0591D990D1120D2D08B9040E7D
:10740000151E0591D990D1120D2D08B9080E191E1F
:107410000591D990D1120D2D08B9A395AF710591A1
:10742000D990D1120D2D08B9A32BF0010591D99057
:10743000D1120D2D08B9CC900591D990D1120D2DF6
:1074400008B9C29E0591D990D1120D2D08B9040E2C
:10745000151E0591D990D1120D2D08B9080E191ECF
:107460000591D990D1120D2D08B9A395AF71059151
:10747000D990D1120D2D08B9A32BF0010591D99007
:10748000D1120D2D08B9CC900591D990D1120D2DA6
:1074900008B9C29E0591D990D1120D2D08B9040EDC
:1074A000151E0591D990D1120D2D08B9080E191E7F
:1074B0000591D990D1120D2D08B9A395AF71059101
:1074C000D990D1120D2D08B9A32BF0010591D990B7
:1074D000D1120D2D08B9CC900591D990D1120D2D56
:1074E00008B9C29E0591D990D1120D2D08B9040E8C
:1074F000151E0591D990D1120D2D08B9080E191E2F
:107500000591D990D1120D2D08B9A395AF710591B0
:10751000D990D1120D2D08B9A32BF0010591D99066
:10752000D1120D2D08B9CC900591D990D1120D2D05
:1075300008B9C29E0591D990D1120D2D08B9040E3B
:10754000151E0591D990D1120D2D08B9080E191EDE
:107550000591D990D1120D2D08B9A395AF71059160
:10756000D990D1120D2D08B9A32BF0010591D99016
:10757000D1120D2D08B9CC900591D990D1120D2DB5
:1075800008B9C29E0591D990D1120D2D08B9040EEB
:10759000151E0591D990D1120D2D08B9080E191E8E
:1075A0000591D990D1120D2D08B9A395AF71059110
:1075B000D990D1120D2D08B9A32BF0010591D990C6
:1075C000D1120D2D08B9CC900591D990D1120D2D65
:1075D00008B9C29E0591D990D1120D2D08B9040E9B
:1075E000151E0591D990D1120D2D08B9080E191E3E
:1075F0000591D990D1120D2D08B9A395AF710591C0
:10760000D990D1120D2D08B9A32BF0010591D99075
:10761000D1120D2D08B9CC900591D990D1120D2D14
:1076200008B9C29E0591D990D1120D2D08B9040E4A
:10763000151E0591D990D1120D2D08B9080E191EED
:107640000591D990D1120D2D08B9A395AF7105916F
:10765000D990D1120D2D08B9A32BF0010591D99025
:10766000D1120D2D08B9CC900591D990D1120D2DC4
:1076700008B9C29E0591D990D1120D2D08B9040EFA
:10768000151E0591D990D1120D2D08B9080E191E9D
:107690000591D990D1120D2D08B9A395AF7105911F
:1076A000D990D1120D2D08B9A32BF0010591D990D5
:1076B000D1120D2D08B9CC900591D990D1120D2D74
:1076C00008B9C29E0591D990D1120D2D08B9040EAA
:1076D000151E0591D990D1120D2D08B9080E191E4D
:1076E0000591D990D1120D2D08B9A395AF710591CF
:1076F000D990D1120D2D08B9A32BF0010591D99085
:10770000D1120D2D08B9CC900591D990D1120D2D23
:1077100008B9C29E0591D990D1120D2D08B9040E59
:10772000151E0591D990D1120D2D08B9080E191EFC
:107730000591D990D1120D2D08B9A395AF7105917E
:10774000D990D1120D2D08B9A32BF0010591D99034
:10775000D1120D2D08B9CC900591D990D1120D2DD3
:1077600008B9C29E0591D990D1120D2D08B9040E09
:10777000151E0591D990D1120D2D08B9080E191EAC
:107780000591D990D1120D2D08B9A395AF7105912E
:10779000D990D1120D2D08B9A32BF0010591D990E4
:1077A000D1120D2D08B9CC900591D990D1120D2D83
:1077B00008B9C29E0591D990D1120D2D08B9040EB9
:1077C000151E0591D990D1120D2D08B9080E191E5C
:1077D0000591D990D1120D2D08B9A395AF710591DE
:1077E000D990D1120D2D08B9A32BF0010591D99094
:1077F000D1120D2D08B9CC900591D990D1120D2D33
:1078000008B9C29E0591D990D1120D2D08B9040E68
:10781000151E0591D990D1120D2D08B9080E191E0B
:107820000591D990D1120D2D08B9A395AF7105918D
:10783000D990D1120D2D08B9A32BF0010591D99043
:10784000D1120D2D08B9CC900591D990D1120D2DE2
:1078500008B9C29E0591D990D1120D2D08B9040E18
:10786000151E0591D990D1120D2D08B9080E191EBB
:107870000591D990D1120D2D08B9A395AF7105913D
:10788000D990D1120D2D08B9A32BF0010591D990F3
:10789000D1120D2D08B9CC900591D990D1120D2D92
:1078A00008B9C29E0591D990D1120D2D08B9040EC8
:1078B000151E0895F0013496CC90C29E040E151E3C
:1078C000080E191E00C00591D990D1120D2D08B9CE
:1078D000A395AF710591D990D1120D2D08B9A32BA5
:1078E000F0010591D990D1120D2D08B9CC900591D8
:1078F000D990D1120D2D08B9C29E0591D990D112FF
:107900000D2D08B9040E151E0591D990D1120D2D1B
:1079100008B9080E191E0591D990D1120D2D08B97C
:10792000A395AF710591D990D1120D2D08B9A32B54
:10793000F0010591D990D1120D2D08B9CC90059187
:10794000D990D1120D2D08B9C29E0591D990D112AE
:107950000D2D08B9040E151E0591D990D1120D2DCB
:1079600008B9080E191E0591D990D1120D2D08B92C
:10797000A395AF710591D990D1120D2D08B9A32B04
:10798000F0010591D990D1120D2D08B9CC90059137
:10799000D990D1120D2D08B9C29E0591D990D1125E
:1079A0000D2D08B9040E151E0591D990D1120D2D7B
:1079B00008B9080E191E0591D990D1120D2D08B9DC
:1079C000A395AF710591D990D1120D2D08B9A32BB4
:1079D000F0010591D990D1120D2D08B9CC900591E7
:1079E000D990D1120D2D08B9C29E0591D990D1120E
:1079F0000D2D08B9040E151E0591D990D1120D2D2B
:107A000008B9080E191E0591D990D1120D2D08B98B
:107A1000A395AF710591D990D1120D2D08B9A32B63
:107A2000F0010591D990D1120D2D08B9CC90059196
:107A3000D990D1120D2D08B9C29E0591D990D112BD
:107A40000D2D08B9040E151E0591D990D1120D2DDA
:107A500008B9080E191E0591D990D1120D2D08B93B
:107A6000A395AF710591D990D1120D2D08B9A32B13
:107A7000F0010591D990D1120D2D08B9CC90059146
:107A8000D990D1120D2D08B9C29E0591D990D1126D
:107A90000D2D08B9040E151E0591D990D1120D2D8A
:107AA00008B9080E191E0591D990D1120D2D08B9EB
:107AB000A395AF710591D990D1120D2D08B9A32BC3
:107AC000F0010591D990D1120D2D08B9CC900591F6
:107AD000D990D1120D2D08B9C29E0591D990D1121D
:107AE0000D2D08B9040E151E0591D990D1120D2D3A
:107AF00008B9080E191E0591D990D1120D2D08B99B
:107B0000A395AF710591D990D1120D2D08B9A32B72
:107B1000F0010591D990D1120D2D08B9CC900591A5
:107B2000D990D1120D2D08B9C29E0591D990D112CC
:107B30000D2D08B9040E151E0591D990D1120D2DE9
:107B400008B9080E191E0591D990D1120D2D08B94A
:107B5000A395AF710591D990D1120D2D08B9A32B22
:107B6000F0010591D990D1120D2D08B9CC90059155
:107B7000D990D1120D2D08B9C29E0591D990D1127C
:107B80000D2D08B9040E151E0591D990D1120D2D99
:107B900008B9080E191E0591D990D1120D2D08B9FA
:107BA000A395AF710591D990D1120D2D08B9A32BD2
:107BB000F0010591D990D1120D2D08B9CC90059105
:107BC000D990D1120D2D08B9C29E0591D990D1122C
:107BD0000D2D08B9040E151E0591D990D1120D2D49
:107BE00008B9080E191E0591D990D1120D2D08B9AA
:107BF000A395AF710591D990D1120D2D08B9A32B82
:107C0000F0010591D990D1120D2D08B9CC900591B4
:107C1000D990D1120D2D08B9C29E0591D990D112DB
:107C20000D2D08B9040E151E0591D990D1120D2DF8
:107C300008B9080E191E0591D990D1120D2D08B959
:107C4000A395AF710591D990D1120D2D08B9A32B31
:107C5000F0010591D990D1120D2D08B9CC90059164
:107C6000D990D1120D2D08B9C29E0591D990D1128B
:107C70000D2D08B9040E151E0591D990D1120D2DA8
:107C800008B9080E191E0591D990D1120D2D08B909
:107C9000A395AF710591D990D1120D2D08B9A32BE1
:107CA000F0010591D990D1120D2D08B9CC90059114
:107CB000D990D1120D2D08B9C29E0591D990D1123B
:107CC0000D2D08B9040E151E0591D990D1120D2D58
:107CD00008B9080E191E0591D990D1120D2D08B9B9
:107CE000A395AF710591D990D1120D2D08B9A32B91
:107CF000F0010591D990D1120D2D08B9CC900591C4
:107D0000D990D1120D2D08B9C29E0591D990D112EA
:107D10000D2D08B9040E151E0591D990D1120D2D07
:107D200008B9080E191E0591D990D1120D2D08B968
:107D3000A395AF710591D990D1120D2D08B9A32B40
:107D4000F0010591D990D1120D2D08B9CC90059173
:107D5000D990D1120D2D08B9C29E0591D990D1129A
:107D60000D2D08B9040E151E0591D990D1120D2DB7
:107D700008B9080E191E0591D990D1120D2D08B918
:107D8000A395AF710591D990D1120D2D08B9A32BF0
:107D9000F0010591D990D1120D2D08B9CC90059123
:107DA000D990D1120D2D08B9C29E0591D990D1124A
:107DB0000D2D08B9040E151E0591D990D1120D2D67
:107DC00008B9080E191E0591D990D1120D2D08B9C8
:107DD000A395AF710591D990D1120D2D08B9A32BA0
:107DE000F0010591D990D1120D2D08B9CC900591D3
:107DF000D990D1120D2D08B9C29E0591D990D112FA
:107E00000D2D08B9040E151E0591D990D1120D2D16
:107E100008B9080E191E0591D990D1120D2D08B977
:107E2000A395AF710591D990D1120D2D08B9A32B4F
:107E3000F0010591D990D1120D2D08B9CC90059182
:107E4000D990D1120D2D08B9C29E0591D990D112A9
:107E50000D2D08B9040E151E0591D990D1120D2DC6
:107E600008B9080E191E0591D990D1120D2D08B927
:107E7000A395AF710591D990D1120D2D08B9A32BFF
:107E8000F0010591D990D1120D2D08B9CC90059132
:107E9000D990D1120D2D08B9C29E0591D990D11259
:107EA0000D2D08B9040E151E0591D990D1120D2D76
:107EB00008B9080E191E0591D990D1120D2D08B9D7
:107EC000A395AF710591D990D1120D2D08B9A32BAF
:107ED000F0010591D990D1120D2D08B9CC900591E2
:107EE000D990D1120D2D08B9C29E0591D990D11209
:107EF0000D2D08B9040E151E0591D990D1120D2D26
:107F000008B9080E191E0591D990D1120D2D08B986
:107F1000A395AF710591D990D1120D2D08B9A32B5E
:107F2000F0010591D990D1120D2D08B9CC90059191
:107F3000D990D1120D2D08B9C29E0591D990D112B8
:107F40000D2D08B9040E151E0591D990D1120D2DD5
:107F500008B9080E191E0591D990D1120D2D08B936
:107F6000A395AF710591D990D1120D2D08B9A32B0E
:107F7000F0010591D990D1120D2D08B9CC90059141
:107F8000D990D1120D2D08B9C29E0591D990D11268
:107F90000D2D08B9040E151E0591D990D1120D2D85
:107FA00008B9080E191E0895F0013596CC90C29EAE
:107FB000040E151E080E191EA395AF710591D990D8
:107FC000D1120D2D08B9A32BF0010591D990D11232
:107FD0000D2D08B9CC900591D990D1120D2D08B96D
:107FE000C29E0591D990D1120D2D08B9040E151E0F
:107FF0000591D990D1120D2D08B9080E191E0591C1
:10800000D990D1120D2D08B9A395AF710591D990D2
:10801000D1120D2D08B9A32BF0010591D990D112E1
:108020000D2D08B9CC900591D990D1120D2D08B91C
:10803000C29E0591D990D1120D2D08B9040E151EBE
:108040000591D990D1120D2D08B9080E191E059170
:10805000D990D1120D2D08B9A395AF710591D99082
:10806000D1120D2D08B9A32BF0010591D990D11291
:108070000D2D08B9CC900591D990D1120D2D08B9CC
:10808000C29E0591D990D1120D2D08B9040E151E6E
:108090000591D990D1120D2D08B9080E191E059120
:1080A000D990D1120D2D08B9A395AF710591D99032
:1080B000D1120D2D08B9A32BF0010591D990D11241
:1080C0000D2D08B9CC900591D990D1120D2D08B97C
:1080D000C29E0591D990D1120D2D08B9040E151E1E
:1080E0000591D990D1120D2D08B9080E191E0591D0
:1080F000D990D1120D2D08B9A395AF710591D990E2
:10810000D1120D2D08B9A32BF0010591D990D112F0
:108110000D2D08B9CC900591D990D1120D2D08B92B
:10812000C29E0591D990D1120D2D08B9040E151ECD
:108130000591D990D1120D2D08B9080E191E05917F
:10814000D990D1120D2D08B9A395AF710591D99091
:10815000D1120D2D08B9A32BF0010591D990D112A0
:108160000D2D08B9CC900591D990D1120D2D08B9DB
:10817000C29E0591D990D1120D2D08B9040E151E7D
:108180000591D990D1120D2D08B9080E191E05912F
:10819000D990D1120D2D08B9A395AF710591D99041
:1081A000D1120D2D08B9A32BF0010591D990D11250
:1081B0000D2D08B9CC900591D990D1120D2D08B98B
:1081C000C29E0591D990D1120D2D08B9040E151E2D
:1081D0000591D990D1120D2D08B9080E191E0591DF
:1081E000D990D1120D2D08B9A395AF710591D990F1
:1081F000D1120D2D08B9A32BF0010591D990D11200
:108200000D2D08B9CC900591D990D1120D2D08B93A
:10821000C29E0591D990D1120D2D08B9040E151EDC
:108220000591D990D1120D2D08B9080E191E05918E
:10823000D990D1120D2D08B9A395AF710591D990A0
:10824000D1120D2D08B9A32BF0010591D990D112AF
:108250000D2D08B9CC900591D990D1120D2D08B9EA
:10826000C29E0591D990D1120D2D08B9040E151E8C
:108270000591D990D1120D2D08B9080E191E05913E
:10828000D990D1120D2D08B9A395AF710591D99050
:10829000D1120D2D08B9A32BF0010591D990D1125F
:1082A0000D2D08B9CC900591D990D1120D2D08B99A
:1082B000C29E0591D990D1120D2D08B9040E151E3C
:1082C0000591D990D1120D2D08B9080E191E0591EE
:1082D000D990D1120D2D08B9A395AF710591D99000
:1082E000D1120D2D08B9A32BF0010591D990D1120F
:1082F0000D2D08B9CC900591D990D1120D2D08B94A
:10830000C29E0591D990D1120D2D08B9040E151EEB
:108310000591D990D1120D2D08B9080E191E05919D
:10832000D990D1120D2D08B9A395AF710591D990AF
:10833000D1120D2D08B9A32BF0010591D990D112BE
:108340000D2D08B9CC900591D990D1120D2D08B9F9
:10835000C29E0591D990D1120D2D08B9040E151E9B
:108360000591D990D1120D2D08B9080E191E05914D
:10837000D990D1120D2D08B9A395AF710591D9905F
:10838000D1120D2D08B9A32BF0010591D990D1126E
:108390000D2D08B9CC900591D990D1120D2D08B9A9
:1083A000C29E0591D990D1120D2D08B9040E151E4B
:1083B0000591D990D1120D2D08B9080E191E0591FD
:1083C000D990D1120D2D08B9A395AF710591D9900F
:1083D000D1120D2D08B9A32BF0010591D990D1121E
:1083E0000D2D08B9CC900591D990D1120D2D08B959
:1083F000C29E0591D990D1120D2D08B9040E151EFB
:108400000591D990D1120D2D08B9080E191E0591AC
:10841000D990D1120D2D08B9A395AF710591D990BE
:10842000D1120D2D08B9A32BF0010591D990D112CD
:108430000D2D08B9CC900591D990D1120D2D08B908
:10844000C29E0591D990D1120D2D08B9040E151EAA
:108450000591D990D1120D2D08B9080E191E05915C
:10846000D990D1120D2D08B9A395AF710591D9906E
:10847000D1120D2D08B9A32BF0010591D990D1127D
:108480000D2D08B9CC900591D990D1120D2D08B9B8
:10849000C29E0591D990D1120D2D08B9040E151E5A
:1084A0000591D990D1120D2D08B9080E191E05910C
:1084B000D990D1120D2D08B9A395AF710591D9901E
:1084C000D1120D2D08B9A32BF0010591D990D1122D
:1084D0000D2D08B9CC900591D990D1120D2D08B968
:1084E000C29E0591D990D1120D2D08B9040E151E0A
:1084F0000591D990D1120D2D08B9080E191E0591BC
:10850000D990D1120D2D08B9A395AF710591D990CD
:10851000D1120D2D08B9A32BF0010591D990D112DC
:108520000D2D08B9CC900591D990D1120D2D08B917
:10853000C29E0591D990D1120D2D08B9040E151EB9
:108540000591D990D1120D2D08B9080E191E05916B
:10855000D990D1120D2D08B9A395AF710591D9907D
:10856000D1120D2D08B9A32BF0010591D990D1128C
:108570000D2D08B9CC900591D990D1120D2D08B9C7
:10858000C29E0591D990D1120D2D08B9040E151E69
:108590000591D990D1120D2D08B9080E191E05911B
:1085A000D990D1120D2D08B9A395AF710591D9902D
:1085B000D1120D2D08B9A32BF0010591D990D1123C
:1085C0000D2D08B9CC900591D990D1120D2D08B977
:1085D000C29E0591D990D1120D2D08B9040E151E19
:1085E0000591D990D1120D2D08B9080E191E0591CB
:1085F000D990D1120D2D08B9A395AF710591D990DD
:10860000D1120D2D08B9A32BF0010591D990D112EB
:108610000D2D08B9CC900591D990D1120D2D08B926
:10862000C29E0591D990D1120D2D08B9040E151EC8
:108630000591D990D1120D2D08B9080E191E05917A
:10864000D990D1120D2D08B9A395AF710591D9908C
:10865000D1120D2D08B9A32BF0010591D990D1129B
:108660000D2D08B9CC900591D990D1120D2D08B9D6
:10867000C29E0591D990D1120D2D08B9040E151E78
:108680000591D990D1120D2D08B9080E191E05912A
:10869000D990D1120D2D08B9A395AF7108952898DE
:1086A0000E94A94BE7E1EA95F1F7289A10D1E0E0A2
:1086B000F6E0F3D0E0FF4ED0E0FF02C00E94C74AD0
:1086C0000895129A0C9464430C94664312984427BC
:1086D0005527662777278CE00C946E430C947043E3
:1086E0000C9472430C9474430C9476430C9478432A
:1086F000440F551F00994160660F771F0199616013
:10870000139A0C9483430C94854313980C948843D8
:108710000C948A430C948C430C948E438A9541F7B5
:1087200040955095609570955F707F704093010CF7
:108730005093020C6093030C7093040C9BE0483040
:10874000590711F40E9480456830790711F40E949E
:1087500080450895EF93E091FB0BE53EE0F5E531B0
:10876000D0F12F923F924F925F926F927F928F92B1
:108770009F92AF92BF92CF92DF92EF92FF920F93B0
:108780001F932F933F934F935F936F937F938F9399
:108790009F93AF93BF93CF93DF930E94082DDF91F8
:1087A000CF91BF91AF919F918F917F916F915F9189
:1087B0004F913F912F911F910F91FF90EF90DF907C
:1087C000CF90BF90AF909F908F907F906F905F9071
:1087D0004F903F902F90EF910895FF93EF93EFB755
:1087E000EF93E0918400EE50E13000F0E23000F0D1
:1087F000E33000F0E43000F0E53000F0E63000F067
:10880000E73000F0E83000F0E93000F005D0EF91FB
:10881000EFBFEF91FF9118950F921F92E8E0FAE5F4
:108820000090FA0B000C1124E00DF11D059014903E
:10883000F00109951F900F90089528980E94A94B68
:10884000E5E1EA95F1F7E091FB0BEA95E093FB0B8C
:10885000289A00000000089528980E94D24B289A78
:108860000000E1E0F6E019D02BD0089528980E948E
:10887000D24BE0EB0000EA95E9F700000000289AEF
:10888000F6E0E2E00AD0089528980E94D24B289A98
:108890000000E3E0FDEF01D008950090FB0B0A9487
:1088A00010905F0011FC0F2E0092FB0B0090FA0B52
:1088B00011FC0E2E0092FA0BE0E011FCE1E00895AD
:1088C000E3E0E0938900EDE8E09388000895E7E0B5
:1088D000E0938900EBE1E09388000895E0EEF4E096
:1088E000A0ECB1E066276D933197E9F71124089564
:1088F0009927772720E2629F080E191EA0ECB1E0AD
:10890000A00DB11D4C93112408950895992720E2DC
:10891000629F080E191EA0ECB1E0A00DB11D509190
:10892000000C450F4C93112408958093000C08957A
:108930008093E10708958093E2079093E3070895F9
:10894000EF92FF920F931F93CF93DF93E0E0F7E056
:1089500020E0822F60814181EF93FF932F930E944B
:10896000AD512F91FF91EF913F9623952F3088F3D2
:1089700055272FE0662775E084EE97E0E0E0F7E00A
:1089800030854281EC01579FC00DD11D540F442307
:1089900049F0317039F069936993699369936993E8
:1089A0004A95C9F73F962A9559F731E02091E1079A
:1089B000213011F43091F90B00EA16E0780123E040
:1089C000A5E0B0E241E0F701329FE00DF11D00812A
:1089D00011811030E9F1183DD8F50030C9F10A389D
:1089E000B8F560E0712F760F783068F1783D58F572
:1089F0007850EC017A9FC00DD11D0880002021F431
:108A00006B9F030E08821FC00980002021F46B9F1A
:108A1000030E098218C00A80002021F46B9F030E08
:108A20000A8211C00B80002021F46B9F030E0B8281
:108A30000AC00C80002039F46B9F030E0C82032EB9
:108A40000A940092F90B259673956395683050F25D
:108A50003395303208F031E04395403208F4B3CF1B
:108A60007091F90B703208F071E07093F90B552793
:108A70002FE0662775E0E0E0F7E030854281EC0109
:108A8000579FC00DD11D540F442349F0317039F464
:108A9000699369936993699369934A95C9F73F9676
:108AA0002A9559F71124DF91CF911F910F91FF90D3
:108AB000EF9008958093FE0B9093FF0B08958091A3
:108AC000FC0B089511241092FC0B0895882329F4BF
:108AD0008091010C9091020C08958091030C90916B
:108AE000040C089580E891E0809361009093610008
:108AF000089580E890E0809361009093610008956C
:108B000028E088E190E00FB6F894A8958093600083
:108B10000FBE2093600008950F931F9303E318E0A6
:108B2000C8010E94274680E790E090930607809353
:108B300005070E946E448FE090E00E948053C801B8
:108B40000E94274641E06FEF80E00E94A54900ECBB
:108B500017E0A8016CE088E00E94335383E090E0C6
:108B60000E94805344EF57E06CE088E00E9433534A
:108B700082E090E00E948053A8016CE088E00E94AF
:108B8000335380E590E00E9480530E946E4484E15C
:108B900090E00E9480531F910F91089590E025E18D
:108BA00030E0829FF001839FF00D929FF00D112421
:108BB000E159F14F618708956093510E089590E057
:108BC00025E130E0829FF001839FF00D929FF00D30
:108BD0001124E159F14F12861182089590E025E1A8
:108BE00030E0829FF001839FF00D929FF00D1124E1
:108BF000E159F14F81E0828B089590E025E130E06A
:108C0000829FF001839FF00D929FF00D1124E15996
:108C1000F14F6087089590E025E130E0829FF001F8
:108C2000839FF00D929FF00D1124E159F14F648361
:108C3000089590E025E130E0829FF001839FF00DE0
:108C4000929FF00D1124E159F14F6583089590939F
:108C5000C60E8093C50E8FE68093CB0E1092200C2B
:108C6000EFE6FEE021E09FEF88E120831782968304
:108C700013861182858375963EE0E33CF307A9F7DE
:108C800008951092700E1092850E10929A0E109206
:108C9000AF0E01969093CF0E8093CE0E90936E0EF2
:108CA00080936D0E9093D20E8093D10E1092CD0EC4
:108CB0001092CC0E1092C40E1092C30E1092C70EDA
:108CC00081E08093200C1092CA0E1092C90E089574
:108CD00080916D0E90916E0E0E9441460895809194
:108CE000780E87FD03C08AEF8093780E80918D0EF9
:108CF00087FD03C08AEF80938D0E8091A20E87FDC1
:108D000003C08AEF8093A20E8091B70E87FD03C047
:108D10008AEF8093B70E1092200C089581E0809323
:108D2000200C0895DC01ED91FC911197AF014F5F8C
:108D30005F4F11965C934E93E4912E2F30E0E7FF46
:108D400013C02F7730703695322F2227379527950D
:108D5000FA014F5F5F4FE4918E2F8F77280F311DFF
:108D6000E7FDF1CF4D935C93C90108958093CB0E3D
:108D7000089508950E949F4A0895EF92FF920F93DD
:108D80001F93CF93DF93182F062FF42EE22EC82FB8
:108D9000D0E085E190E0C89FF001C99FF00DD89F19
:108DA000F00D1124E159F14F8285882321F0818152
:108DB000882309F087C0EE2091F485E190E0C89FF8
:108DC000F001C99FF00DD89FF00D1124E159F14F2A
:108DD000128A8185882309F075C0178273C0133009
:108DE00059F481E091E09093530E8093520E81E00C
:108DF0008093510E0F2D08C060E0812F0E949F4A82
:108E00006F2D812F0E94804A0F3799F485E190E001
:108E1000C89FF001C99FF00DD89FF00D1124E159B2
:108E2000F14F8091C80E868789EC9EE0948B838BEE
:108E300030C089E0089FC0011124E091C50EF09177
:108E4000C60EE80FF91F339645915491411551050F
:108E500071F485E190E0C89FF001C99FF00DD89FA3
:108E6000F00D1124E159F14F148A138A12C0FA014E
:108E7000249185E190E0C89FF001C99FF00DD89F33
:108E8000F00D1124E159F14F26874F5F5F4F548B4E
:108E9000438B85E190E0C89FF001C99FF00DD89FFA
:108EA000F00D1124E159F14F1786118603871182C5
:108EB0008FEF8087E782F282108A81E08287128AB0
:108EC000118A1482DF91CF911F910F91FF90EF9043
:108ED0000895CF92DF92FF920F931F93CF93DF936A
:108EE000E7E7FEE08181282F332727FD3095808139
:108EF000280F311D2F3F310519F014F02FEF30E00E
:108F0000C90137FF02C080E090E0808375964EE093
:108F1000EB3CF40739F78091200C882309F019C144
:108F200035C1E091CE0EF091CF0E9F012F5F3F4FE4
:108F30003093CF0E2093CE0E44914F3F69F5A90197
:108F40004F5F5F4F5093CF0E4093CE0EF901849147
:108F50008F3219F41092200C0AC1863009F0EAC051
:108F6000FA013196CF0101969093CF0E8093CE0EE9
:108F7000E491E33529F49093D20E8093D10EDAC0B8
:108F8000E53409F0D7C08091D10E9091D20E909324
:108F9000CF0E8093CE0ECEC047FF02C04093C70EC7
:108FA000542F5F70842F90E0807F9070803B9105FC
:108FB00029F1803C910579F18039910509F042C091
:108FC000C9010196F901449101969093CF0E8093C7
:108FD000CE0E0197FC012491852F90E08C9FF0012B
:108FE0008D9FF00D9C9FF00D1124E159F14F808170
:108FF000882309F49FC0220F638552C0C9010196DE
:10900000F901449101969093CF0E8093CE0E019773
:10901000FC01249153C02F5F3F4F3093CF0E20931C
:10902000CE0E21503040F9012491852F90E08C9F85
:10903000F0018D9FF00D9C9FF00D1124E159F14F2F
:10904000238778C08091C70E582F5F7090E0807F93
:109050009070803B910541F1803C910509F45EC020
:109060008039910509F066C02F5F3F4F3093CF0ED6
:109070002093CE0E21503040F9012491852F90E0AD
:109080008C9FD0018D9FB00D9C9FB00D1124A159D4
:10909000B14F8C91882309F44DC0220F1B966C911F
:1090A000852F0E94BD4646C02F5F3F4F3093CF0EA5
:1090B0002093CE0E21503040F9012491473071F4B5
:1090C000852F90E08C9FF0018D9FF00D9C9FF00DFF
:1090D0001124E159F14F220F26832CC04C3571F435
:1090E000852F90E08C9FF0018D9FF00D9C9FF00DDF
:1090F0001124E159F14F220F24831CC04436D1F4CE
:10910000852F90E08C9FF0018D9FF00D9C9FF00DBE
:109110001124E159F14F220F25830CC0852F90E0D7
:109120008C9FF0018D9FF00D9C9FF00D1124E15953
:10913000F14F43878EEC9EE00E949246969587956C
:109140009093CD0E8093CC0E1092C40E1092C30E4D
:1091500002C0C5E1D0E06091C30E7091C40E809151
:10916000CC0E9091CD0E6817790709F4DACE6F5FB7
:109170007F4F7093C40E6093C30E8091C90E90917F
:10918000CA0E01969093CA0E8093C90E02E31EE0A8
:10919000C0E7DEE0FF24BFEFCB2ED12C89898823E6
:1091A00009F05EC08A899B89892B09F456C09E8587
:1091B0008D85981708F04CC050C08A852A893B8954
:1091C0008F37E9F4D9018D91BB8BAA8B8F3F01F1C9
:1091D000F90161811196BB8BAA8BE82FF0E0EE0FAD
:1091E000FF1FE45CF74F0190F081E02D8F2D099572
:1091F000EA89FB8981918D87FB8BEA8B28C0A901C5
:109200004F5F5F4F5B8B4A8BF90184918F3F21F455
:1092100018821B8A1A8A21C04F5F5F4F5B8B4A8B73
:1092200041505040FA01649190E0880F991F845C8E
:10923000974FFC01259134918F2DF9010995EA8909
:10924000FB893196FB8BEA8B3197E491ED871E8683
:109250009E858D85981709F4B0CF8E858F5F8E8798
:109260008985882319F420E030E05DC08F858F3F29
:1092700011F08F5F8F879E81992309F44EC02F8153
:10928000222309F44AC08D81882309F446C0409105
:10929000CB0E442309F441C0899FC00111248050A2
:1092A0009F4F892F992730E0BC01629FC001639FC7
:1092B000900D729F900D112480509F4F892F9927F8
:1092C000242F30E0FC01E29FC001E39F900DF29F4C
:1092D000900D112480509F4F292F33278B81882395
:1092E000F1F0EA81F0E0E050F846E491E058E89FC0
:1092F000C001112480509F4F892F9927A601481B38
:10930000590B429FC001439F900D529F900D112415
:1093100080509F4F292F332702C020E030E08A8100
:109320009C81890F8A83F8012083F394065F1F4F85
:109330006596F4E0FF1609F031CFDF91CF911F91D0
:109340000F91FF90DF90CF9008951F93CF93DF93FD
:10935000582F89E0589FC00111242091C50E3091EB
:10936000C60E280F391FC9010396FC01A591B491BF
:10937000F90184918150823010F413E01DC0809176
:10938000850E8823B1F08091900E851711F4442347
:1093900081F480919A0E882371F08091A50E851733
:1093A00011F4442341F49091940E8091A90E8917F1
:1093B00010F411E001C012E0212F30E0FD014491D2
:1093C00085E190E0289FE001299FD00D389FD00DC6
:1093D0001124C159D14F4E871196BC8BAB8B1F8680
:1093E00080E58A836F838FEF888719861A8A188AA7
:1093F00021E02A87198A5C8729831C82133049F46B
:1094000081E091E09093530E8093520E2093510E81
:1094100008C060E5812F0E94804A6989812F0E94DF
:109420009F4ADF91CF911F910895FF920F931F9351
:10943000082FF62E0E94804A10E085E190E0089FF8
:10944000F001099FF00D189FF00D1124E159F14F23
:10945000F2821F910F91FF900895962F482F50E0B0
:1094600025E130E0429FF001439FF00D529FF00D47
:109470001124E159F14F6281691B62830E94804A85
:109480000895482F50E025E130E0429FF001439FCE
:10949000F00D529FF00D1124E159F14F9281690FA7
:1094A00062830E94804A08950000000000000000CE
:1094B00000000000000000000000000000000000AC
:1094C000000000000000000000000000000000009C
:1094D000000000000000000000000000000000008C
:1094E000000000000000000000000000000000007C
:1094F000000000000000000000000000000000006C
:1095000099277727833008F00895E0E0F2EA660FA4
:10951000771FE60FF71FA591B491E2E3FEE02AE082
:10952000289FE00DF11DA183B2831124089590912D
:10953000510E9170880F892B8093510E08959927B1
:109540007727E2E3FEE02AE0289FE00DF11D6E3F61
:1095500031F46091510E6E7F6093510E0BC06F3FDE
:1095600031F46091510E6E6F6093510E03C078E933
:10957000760F75831124089599277727E2E3FEE09B
:109580002AE0289FE00DF11D6083112408952F9398
:109590003F934F935F936F937F938F939F93AF937B
:1095A000BF93789411240E94A0440E9461430E94BA
:1095B00069472F923F924F925F926F927F928F9264
:1095C0009F92AF92BF92CF92DF92EF92FF920F9352
:1095D0001F93CF93DF9300902F0E002019F4A1E288
:1095E000BCE002C0A7E2BDE001E0002600922F0E21
:1095F00002E00093300E5091500E6091520E709127
:10960000530E8091540E2090330E3090340E4090C3
:10961000360E5090370E6090350E1091320E7090CD
:109620003D0E80903E0E90903F0EA090400EB09068
:10963000410E20913C0EC090470ED090480EE09015
:109640004A0EF0904B0E0091490E3091460E9FEF5E
:10965000620C431CF2014491410300240008C12D17
:10966000D02D970CA81CF50144914203002400085A
:10967000C10DD01D0C0DED1CF701449143030024D6
:109680000008C10DD01D8A956AF44091510E842FB7
:109690008695062E0694062600FA7695679576F945
:1096A00040FF66F940E860FD4FE7450300240008ED
:1096B000C10DD01D0024C038D0050CF0CFE70A94AE
:1096C000C038D0050CF4C0E8C058CD939A9509F085
:1096D000BFCF4091300E4A954093300E97E009F08D
:1096E000B7CF6092350E4092360E90923F0EA09208
:1096F000400E0093490EE0924A0E6093520E709312
:10970000530E8093540EDF91CF911F910F91FF90D4
:10971000EF90DF90CF90BF90AF909F908F907F9011
:109720006F905F904F903F902F9099278091FA0B08
:1097300077276091FB0B11240E94B946BF91AF912E
:109740009F918F917F916F915F914F913F912F9159
:1097500008950C94AB4B0C94AD4B0F931F932ABD03
:10976000E0912D0EF0912E0E019100000093B300B8
:109770000EE0ED32F00710F40000000010F0E1E21E
:10978000FCE0E0932D0EF0932E0EC895C895C89579
:10979000C895C895C8950000000000002AB51F9123
:1097A0000F9108950000E091FB0BE0FFD6CFE1E1BF
:1097B000EA95F1F7000000000895000000000000A5
:1097C0000000000000000000000000000000000099
:1097D0000000000000000000000000000000000089
:1097E0000000000000000000000000000000000079
:1097F0000000000000000000000000000000000069
:10980000000306090C101316191C1F2225282B2EE5
:10981000313336393C3F414447494C4E51535558FA
:109820005A5C5E60626466686A6B6D6F70717374B7
:10983000757678797A7A7B7C7D7D7E7E7E7F7F7F70
:109840007F7F7F7F7E7E7E7D7D7C7B7A7A79787656
:1098500075747371706F6D6B6A68666462605E5C6C
:109860005A585553514E4C494744413F3C39363381
:10987000312E2B2825221F1C191613100C09060344
:1098800000FDFAF7F4F0EDEAE7E4E1DEDBD8D5D24B
:10989000CFCDCAC7C4C1BFBCB9B7B4B2AFADABA816
:1098A000A6A4A2A09E9C9A9896959391908F8D8C39
:1098B0008B8A888786868584838382828281818160
:1098C0008181818182828283838485868687888A5A
:1098D0008B8C8D8F9091939596989A9C9EA0A2A424
:1098E000A6A8ABADAFB2B4B7B9BCBFC1C4C7CACDEF
:1098F000CFD2D5D8DBDEE1E4E7EAEDF0F4F7FAFD0C
:10990000808182838485868788898A8B8C8D8E8FDF
:10991000909192939495969798999A9B9C9D9E9FCF
:10992000A0A1A2A3A4A5A6A7A8A9AAABACADAEAFBF
:10993000B0B1B2B3B4B5B6B7B8B9BABBBCBDBEBFAF
:10994000C0C1C2C3C4C5C6C7C8C9CACBCCCDCECF9F
:10995000D0D1D2D3D4D5D6D7D8D9DADBDCDDDEDF8F
:10996000E0E1E2E3E4E5E6E7E8E9EAEBECEDEEEF7F
:10997000F0F1F2F3F4F5F6F7F8F9FAFBFCFDFEFF6F
:10998000000102030405060708090A0B0C0D0E0F5F
:10999000101112131415161718191A1B1C1D1E1F4F
:1099A000202122232425262728292A2B2C2D2E2F3F
:1099B000303132333435363738393A3B3C3D3E3F2F
:1099C000404142434445464748494A4B4C4D4E4F1F
:1099D000505152535455565758595A5B5C5D5E5F0F
:1099E000606162636465666768696A6B6C6D6E6FFF
:1099F000707172737475767778797A7B7C7D7E7FEF
:109A000000020406080A0C0E10121416181A1C1E66
:109A100020222426282A2C2E30323436383A3C3E56
:109A200040424446484A4C4E50525456585A5C5E46
:109A300060626466686A6C6E70727476787A7C7E36
:109A40007F7D7B79777573716F6D6B696765636116
:109A50005F5D5B59575553514F4D4B494745434106
:109A60003F3D3B39373533312F2D2B2927252321F6
:109A70001F1D1B19171513110F0D0B0907050301E6
:109A8000FFFDFBF9F7F5F3F1EFEDEBE9E7E5E3E1D6
:109A9000DFDDDBD9D7D5D3D1CFCDCBC9C7C5C3C1C6
:109AA000BFBDBBB9B7B5B3B1AFADABA9A7A5A3A1B6
:109AB0009F9D9B99979593918F8D8B8987858381A6
:109AC00080828486888A8C8E90929496989A9C9EA6
:109AD000A0A2A4A6A8AAACAEB0B2B4B6B8BABCBE96
:109AE000C0C2C4C6C8CACCCED0D2D4D6D8DADCDE86
:109AF000E0E2E4E6E8EAECEEF0F2F4F6F8FAFCFE76
:109B00007F7F7F7F7F7F7F7F7F7F7F7F7F7F7F7F65
:109B10007F7F7F7F7F7F7F7F7F7F7F7F7F7F7F7F55
:109B20007F7F7F7F7F7F7F7F7F7F7F7F7F7F7F7F45
:109B30007F7F7F7F7F7F7F7F7F7F7F7F7F7F7F7F35
:109E00000309131E28313A40464C5054585B5E619A
:109E1000636567696B6C6E6F70717273747576775A
:109E2000777879797A7A7B7B7C7C7C7D7D7D7E7E80
:109E30007E7E7F7F7F7F7F7F7F7F7F7F7F7F7F7F34
:109E40007F7F7F7F7F7F7F7F7F7F7F7F7F7E7E7E25
:109E50007E7D7D7D7C7C7C7B7B7A7A797978777757
:109E6000767574737271706F6E6C6B696765636120
:109E70005E5B5854504C46403A31281E130903008B
:109E8000C6CCD5DBDFE3E5E7E9EAEBECEDEEEFEF9F
:109E9000F0F0F0F1F1F1F1F2F2F2F2F2F2F2F2F3AB
:109EA000F3F3F3F3F3F3F3F3F3F3F3F3F3F3F3F382
:109EB000F3F3F3F3F3F3F3F3F3F3F3F3F3F3F3F372
:109EC000F3F3F3F3F3F3F3F3F3F3F3F3F3F3F3F362
:109ED000F3F3F3F3F3F3F3F3F3F3F3F3F3F3F3F352
:109EE000F2F2F2F2F2F2F2F2F1F1F1F1F0F0F0EF5F
:109EF000EFEEEDECEBEAE9E7E5E3DFDBD5CCC6001E
:109F000000283D42302D2C2B2C2D2E2F3032333576
:109F100037393B3D3F414345484A4C4E50535557D6
:109F2000595B5D5F61636567696B6C6E70717374BB
:109F3000757778797A7B7C7D7D7E7E7F7F7F7F7F62
:109F40007F7F7F7F7F7F7E7E7D7D7C7B7A79787748
:109F500075747371706E6C6B69676563615F5D5B6F
:109F600059575553504E4C4A484543413F3D3B3964
:109F700037353332302F2E2D2C2B2C2D30423D28CF
:109F800000E9E5FED4D7D7D7D6D4D2D0CECCCAC834
:109F9000C6C3C1BFBDBAB8B6B4B1AFADABA9A7A572
:109FA000A3A19F9E9C9A999795949391908F8D8C45
:109FB0008B8A898888878685858484848383838344
:109FC0008383838383848484858586878888898A3C
:109FD0008B8C8D8F909193949597999A9C9E9FA12D
:109FE000A3A5A7A9ABADAFB1B4B6B8BABDBFC1C345
:109FF000C6C8CACCCED0D2D4D6D7D7D7D4FEE5E9FE
:10A00000F9F8F9F5EBE1DDDEE0E2E4E5E6E5E4E2CE
:10A01000DED9D2CAC1B7ACA299918A8683818080E9
:10A020008182838586888A8C8D8F9092939596976E
:10A0300098999A9B9B9C9D9D9D9E9E9E9F9F9F9F56
:10A040009F9F9F9E9E9E9D9D9D9C9B9B9A9998974E
:10A0500096959392908F8D8C8A8886858382818055
:10A06000808183868A9199A2ACB7C1CAD2D9DEE237
:10A07000E4E5E6E5E4E2E0DEDDE1EBF5F9F8F90040
:10A080000708070B151F2322201E1C1B1A1B1C1E52
:10A0900022272E363F49545E676F767A7E7F7F7F18
:10A0A0007F7E7D7B7A7876747371706E6D6B6A6972
:10A0B0006867666565646463636262626161616169
:10A0C0006161616262626363636465656667686952
:10A0D0006A6B6D6E7071737476787A7B7D7E7F7F2C
:10A0E0007F7F7E7A766F675E54493F362E27221E29
:10A0F0001C1B1A1B1C1E2022231F150B0708070000
:10A100001F313D444E5354565A5F64696E747679DC
:10A110007C7F7F7F7F7F7F7F7F7F7F7F7F7F7F7F52
:10A120007F7F7F7F7F7F7F7F7F7F7F7F7F7F7F7F3F
:10A130007F7F7F7F7F7F7F7F7F7F7F7F7F7F7F7F2F
:10A140007F7F7F7F7F7F7F7F7F7F7F7F7F7F7F7F1F
:10A150007F7F7F7F7F7F7F7F7F7F7F7F7F7F7F7F0F
:10A160007F7F7F7F7F7F7F7F7F7F7F7F7F7F7F7FFF
:10A170007F7F7F7F7F7F7F7F7F7F7F7C7871684C51
:10A180002C1C120C0A0B0A05FDF3E9DFD4CAC0B778
:10A19000AEA69E97918B868582808080808080800D
:10A1A00080808080808080808080808080808080AF
:10A1B000808080808080808080808080808080809F
:10A1C000808080808080808080808080808080808F
:10A1D000808080808080808080808080808080807F
:10A1E000808080808080808080808080808080806F
:10A1F000808080808087919DACC4CBD4DDF2FAFA58
:10A2000022002400260028002B002D0030003300FF
:10A21000360039003D004000440048004C00510029
:10A2200056005B00600066006C00730079008100DE
:10A23000880090009900A200AC00B600C100CC00DC
:10A24000D800E500F30001011001210132014401B1
:10A2500057016C0181019801B001CA01E5010202B8
:10A260002102410264028802AE02D70203033003D6
:10A2700061039403CB03050442048304C70410055F
:10A280005D05AF0505066106C206290796070908A0
:10A29000830805098E09200ABA0A5D0B0A0CC10C55
:10A2A000840D510E2B0F121007110A121D134014AA
:10A2B0007415BA1614188319071BA31C571E2420E3
:10A2C0000E22142439267F28E82A752D29300633DA
:10A2D0000F364539AD3C49401B442848734CFE506D
:10A2E000CF55EA5A51600C661D6C8B725A79928078
:10A2F00037885090E598FDA19FABD3B5A3C000006F
:10A300001F93CF93DF93FA01549131961491C52F87
:10A31000D0E09F012F5F3F4F70E095E0660F771F01
:10A320009A95E1F7680F711D40E00BC084918D9301
:10A330009F5F31969517D0F34F5F2C0F3D1F605EE6
:10A340007F4F411730F4DB01A054BE4FF90190E07C
:10A35000F1CFDF91CF911F910895382F603CD0F459
:10A3600070E0660F771FCB018E5A974FFC01249146
:10A370006D5A774FFB016491832F90E0FC0174E0EC
:10A38000EE0FFF1F7A95E1F7E81BF90BE050F94F4C
:10A3900021876287832F90E0FC0154E0EE0FFF1FBE
:10A3A0005A95E1F7E81BF90BE050F94F81852381BD
:10A3B0003481280F311D3687258746954695469569
:10A3C000842F90E045E0880F991F4A95E1F7280F08
:10A3D000391F3487238708958F929F92AF92BF923F
:10A3E000CF92DF92EF92FF920F931F93CF93DF9361
:10A3F000882E962E5A016901F02E00E010E080EEC2
:10A40000F80E0CC04F2D6E2D882D8C0F0E948644A7
:10A410002196CA15DB05B4F30F5F1F4F0C151D0500
:10A420002CF4C0E0D0E0E02EE90CF3CFDF91CF9127
:10A430001F910F91FF90EF90DF90CF90BF90AF9062
:10A440009F908F90089540520E9486440895FF92F5
:10A450000F931F93CF93DF938C01F62EEA01FE0139
:10A4600044912196442349F0802F0F5F1F4F4F776F
:10A4700040526F2D0E948644F2CFDF91CF911F9101
:10A480000F91FF900895FF920F931F93182F062F9F
:10A49000F42E42954F704A3010F4405F01C0495E7F
:10A4A000602F812F0E9486444F2D4F70812F8F5F28
:10A4B0004A3010F4405F01C0495E602F0E9486441C
:10A4C0001F910F91FF900895FF920F931F93F82E05
:10A4D000162F042F452F0E944352402F612F8F2D9E
:10A4E0008E5F0E9443521F910F91FF900895EF924B
:10A4F000FF920F931F93F62E042F182FF8E0EF2EE4
:10A50000E80E07FF02C041E101C040E16F2D812F3D
:10A510000E9486441F5F1E1511F0000FF2CF1F919D
:10A520000F91FF90EF900895FF920F931F93CF9399
:10A53000DF93F62E042FEC0110E0002311F4112319
:10A5400039F4802F6AE00E944557905F492F01C07F
:10A5500040E06F2D8C2F0E9486441F5F219713309F
:10A5600031F0802F6AE00E944557082FE6CFDF9137
:10A57000CF911F910F91FF900895CF92DF92EF92AC
:10A58000FF920F931F93CF93DF93C62E79018A0119
:10A59000EC01DD24E114F1040105110511F4DD20C5
:10A5A00059F4C801B7012AE030E040E050E00E94D1
:10A5B0005157462F405F01C040E06C2D8C2F0E9408
:10A5C0008644D394219786E0D81669F0C801B70174
:10A5D0002AE030E040E050E00E945157C901DA0122
:10A5E0007C018D01D7CFDF91CF911F910F91FF900B
:10A5F000EF90DF90CF9008957F928F929F92AF92CD
:10A60000BF92CF92DF92EF92FF920F931F93CF935F
:10A61000DF93782E862E5A016901780100E010E060
:10A620000CC0A701692D872D8C0F0E9478442196BC
:10A63000CA15DB05B4F30F5F1F4F0C151D052CF475
:10A64000C0E0D0E0902E980CF3CFDF91CF911F9116
:10A650000F91FF90EF90DF90CF90BF90AF909F90C1
:10A660008F907F9008957F928F929F92AF92BF922A
:10A67000CF92DF92EF92FF920F931F93CF93DF93CE
:10A68000782E862EEA01FA01C590D490FA0132960E
:10A69000A590B49000E016C0FC01EE0DFF1D3296AF
:10A6A000EE0FFF1FEC0FFD1F45915491692D812F77
:10A6B000870D0E9478441F5F812F90E08C159D05C7
:10A6C0005CF30F5F802F90E08A159B055CF48C9DF6
:10A6D00070018D9DF00C9C9DF00C112410E0902ECB
:10A6E000980CEACFDF91CF911F910F91FF90EF90DF
:10A6F000DF90CF90BF90AF909F908F907F90089504
:10A700000F931F93CF93DF938C01C0E0D0E007C07D
:10A710000E945F458823E1F30E9462452196C0179D
:10A72000D107B4F3DF91CF911F910F9108951F933B
:10A73000CF93DF93A091670EB091680EBD01660FB5
:10A74000771FCB018A0F9B1FFC01EA57F74AE49160
:10A75000E35DE093EE06AC014F5F5F4FFA01EA570D
:10A76000F74AE491E35DE093F1069C012E5F3F4FD1
:10A77000F901EA57F74AE491E35DE093F406815763
:10A78000974AFC018491835D8093EF064157574AB5
:10A79000FA014491435D4093F2062157374AF9018B
:10A7A0002491235D2093F506FD01E256F74AE491DA
:10A7B000E85DE093F006FB01E856F74AE491E85DB6
:10A7C000E093F3066756774AFB016491685D6093F6
:10A7D000F6068091690E8F5F8093690E80315CF080
:10A7E0001092690E80916A0E8F5F80936A0E84309A
:10A7F00014F010926A0E8091690E80FF08C0CD019E
:10A8000001969093680E8093670E0397BCF4E091D5
:10A810006A0EFF27E7FDF095EE0FFF1FCF018F5E59
:10A82000984ACEEEDEE0A0EDB6E0E05FF84A549143
:10A83000FC01449110E271E261E005C01092680EE3
:10A840001092670EE4CF8C81882309F43AC08F5FA1
:10A850008C8387FD6C83EC818E2F90E00197FC0147
:10A86000E858F84AE4912E2F30E02C5E3F4F3983B0
:10A8700028838850984AFC01849190E00F96959522
:10A880008795C8969B838A832C9311968C931197F6
:10A890002A5F13962C93139714968C9314978D819B
:10A8A000882339F412961C93129715967C9315976A
:10A8B00008C0813031F412965C93129715964C9330
:10A8C000159727961696FFE0C831DF0709F0BBCF32
:10A8D000DF91CF911F910895E3EDFEE0A8EBB6E084
:10A8E0002FEF3FEF4FEF8481882371F082819381B6
:10A8F00004979383828311968C931197849720F405
:10A900003183208314824C93359613968EE0E73E74
:10A91000F80749F72091ED0E222311F18091E90EFD
:10A920009091EA0E02969093EA0E8093E90E2F5FC3
:10A930002093ED0E8093C706822F63E00E94455757
:10A94000935E9093C906253158F01092ED0E8FEF6B
:10A950009FEF9093EA0E8093E90E8FEF8093C706E6
:10A960000895E7EDFEE040E050E08081882309F0A3
:10A970004EC0DA01AA0FBB1FAA0FBB1FA40FB51F41
:10A98000AD52B14F81E014968C931497E091640E10
:10A990008091A101EE2319F490E0049710C0EF5FBD
:10A9A000E093640EE150F0E0E85CF84AE49190E056
:10A9B00004972E2F332727FD3095820F931F139670
:10A9C0009C938E9312972091A00130E02F5F3F4F10
:10A9D000DA01AA0FBB1FAA0FBB1FA40FB51FAD52F0
:10A9E000B14F11963C932E93CA010896FC01EE0FCD
:10A9F000FF1FE80FF91FE056F94F8CE18283208397
:10AA000012968C9181838AE08093A20107C04F5FE8
:10AA10005F4F35964430510509F0A7CF8091ED0E78
:10AA20008823F9F48091640E8823D9F481E080931F
:10AA3000ED0E2091A10130E0275F3F4F3093EC0EE7
:10AA40002093EB0E8091A00190E042969093EA0E45
:10AA50008093E90E8093C7062093C8068DE180930A
:10AA6000C9060895CF93DF9380E00E946645EC010C
:10AA700083FF07C08091640E882319F481E08093DE
:10AA8000640ED3FF0CC08091650E9091660E93FD0D
:10AA900006C08091A201882311F40E94B154C5FF21
:10AAA0000AC08091A00181508093A001843118F4E4
:10AAB00084E18093A001C4FF0AC08091A0018F5F50
:10AAC0008093A0018E3218F08DE28093A001C2FF26
:10AAD0000BC02FEF47E161E083E00E94BD4680E0BC
:10AAE0000E946645892BD9F7D2FF04C01092B80E98
:10AAF0001092B50ED1FF05C080E00E946645892BFB
:10AB0000D9F7D093660EC093650E80E0DF91CF91A8
:10AB100008955F926F927F928F929F92AF92BF92B1
:10AB2000CF92DF92EF92FF920F931F93DF93CF9319
:10AB30000F92CDB7DEB70E946E4481EE95E50E947C
:10AB4000274680EC0E94B64684E699E30E949B4427
:10AB500080E00E949844E5E0F7E044E65AE0518343
:10AB600040833F9687E0EC38F807C9F780E280938E
:10AB70000207FF24F394F092080784E992E490938B
:10AB800006078093050720E32093110780E492E0F5
:10AB90009093130780931207F092170750931507AD
:10ABA000409314072093200780E093E090932207BE
:10ABB00080932107F09226075093240740932307A0
:10ABC00028E220932F0780EC93E090933107809345
:10ABD0003007F092350784E09FE19093330780932C
:10ABE000320720933E0780E694E0909340078093DD
:10ABF0003F07F092440784EF91E3909342078093DC
:10AC0000410701E010E021E030E040E250E065E281
:10AC100070E080E090E00E94FC5202E010E021E051
:10AC200030E040E250E066E270E080E090E00E94B8
:10AC3000FC524AE059E360E080E00E94805148E421
:10AC400058E36AE080E00E94805146EA57E360E101
:10AC500080E00E94805144E057E365E180E00E947B
:10AC6000805184E19AE40E94414684E18093F20E8F
:10AC700082E38093F90E86E48093000F8AE5809347
:10AC8000070F8EE680930E0FF0920F0F198200E0EF
:10AC9000552453947EE0872E68E1762E50E1652E90
:10ACA00042E0A42E33E0932E24E0B22E90E8F92E59
:10ACB00089E1D82EBAE1CB2EABE1EA2E81E090E01B
:10ACC0000E9480530E946C5480915A0E81FF02C0F2
:10ACD0000E9497538091A201882319F0815080939C
:10ACE000A2010F5F033071F48091620E8F5F809339
:10ACF000620E803C10F01092620E8091620E809382
:10AD00001E0700E0E981E13019F0F1E0F98312C09B
:10AD100080915E0E8F5F80935E0E1150803C10F02C
:10AD200010925E0E112309F410EC80915E0E809358
:10AD30002D07198280915A0E8F5F80935A0E803CA6
:10AD400010F010925A0E30915A0E30933C078091B9
:10AD5000A0018F5F8093A30681508093A606282FC1
:10AD60002A5F2093A906982F945F9093AC06809356
:10AD7000AF062093B2069093B506E091640EEE23E1
:10AD800009F03FC03695232F30E0F901EF71F070E4
:10AD9000E85EF84AE4918091A101E80FE093A406EF
:10ADA0008E2F885F8093A7068093AA068093AD06B6
:10ADB000E05FE093B006E093B306E093B6065092EE
:10ADC000A506A092A8069092AB06B092AE06277098
:10ADD0003070C901880F991F820F931FFC01E85042
:10ADE000F94AE491E093B106FC01E750F94AE49195
:10ADF000E093B4068650994AFC0124912093B7064B
:10AE00002BC03695369541F18092B1067092B4060A
:10AE10006092B7068E2F8F5F8093640EF0E0E85C3F
:10AE2000F84AE491E093E80E803410F01092640E3A
:10AE30008091A1018E0F8093A406982F985F909324
:10AE4000A7069093AA069093AD06805F8093B00604
:10AE50008093B3068093B6061C521093F7061A5FD0
:10AE60001093FA061A5F1093FD06105EF092F80632
:10AE7000F092FB06F092FE06D092F906C092FC0614
:10AE8000E092FF060E94325519CF991B79E004C069
:10AE9000991F961708F0961B881F7A95C9F7809519
:10AEA0000895A1E21A2EAA1BBB1BFD010DC0AA1F0B
:10AEB000BB1FEE1FFF1FA217B307E407F50720F023
:10AEC000A21BB30BE40BF50B661F771F881F991F9E
:10AED0001A9469F760957095809590959B01AC01E7
:0AAEE000BD01CF010895F894FFCFE3
:10AEEA000000000000000000000000000000000058
:10AEFA000000000000000000000000000000000048
:10AF0A000000000000000000000000000000000037
:10AF1A000000000000000000000000000000000027
:10AF2A000000000000000000000000000000000017
:10AF3A000000000000000000000000000000000007
:10AF4A0000000000000000000000000000000000F7
:10AF5A0000000000000000000000000000000000E7
:10AF6A0000000000000000000000000000000000D7
:10AF7A007B2EF1316935E1385A3CD43F3CC3030199
:04AF8A001EA81E00DF
:00000001FF
